:020000040800F2
:10000000C81D00200101000821550008ED3D000831
:1000100065530008C10F00080981000800000000B6
:100020000000000000000000000000008D650008D6
:10003000BB2D000800000000C95A0008B568000880
:100040001B010008855800081B0100081B0100085F
:100050001B0100081B0100081B0100081B01000810
:100060001B0100081B0100081B0100081B01000800
:100070001B0100081B010008E12800081B01000803
:100080001B0100081B01000859070008D97B000864
:10009000857C00081B010008E90F00081B0100080F
:1000A00045690008416A00081B0100081B0100089F
:1000B000456A00082D6D0008896F00081B010008C3
:1000C0001B0100081B0100081B0100081B010008A0
:1000D0001B010008297B00081B0100081B01000808
:1000E0001B0100081B0100081B010008DFF80CD0F1
:1000F00000F0F4FA0048004709970008C81D0020E6
:100100000648804706480047FEE7FEE7FEE7FEE7B1
:10011000FEE7FEE7FEE7FEE7FEE7FEE7D168000840
:10012000ED0000082DE9F0410024061B254671F181
:10013000000605DA01240027D0EB070067EB010178
:10014000161E73F1000605DA0027D2EB070201251F
:1001500067EB030300F0DEF986460E4617469C4621
:10016000AC4204D00025D0EB050E65EB010624B1AE
:100170000020D2EB000760EB030C704631463A4694
:100180006346BDE8F08140EA01039B0703D009E024
:1001900008C9121F08C0042AFAD203E011F8013B73
:1001A00000F8013B521EF9D2704710B5002200E062
:1001B000521C835C8C5CA34201D1002BF8D1D8B2D5
:1001C000E1B2401A10BD80EA010210B502F000430E
:1001D000400022D04A001FD0010E01EB1261C0F393
:1001E0005600C2F3560240F4000042F40002A0FBA5
:1001F000022000047F39140400D0401C50EA124051
:1002000001D44000491EC2B20C0604EBD010401CC1
:100210004008802A02D003E0002010BD20F0010039
:10022000002900DA0020184310BD2DE9FE4F81EAB5
:10023000030404F0004421F0004100944FF0000B4F
:1002400023F0004350EA01045ED052EA03045BD07D
:10025000C3F30A54C1F30A552C44A4F2F3340194B5
:10026000A0FB0254C1F3130141F48011C3F3130343
:1002700043F4801301FB024400FB034E840A970AF7
:1002800044EA815447EA8357A4FB076802958D0A24
:1002900005FB07854FEA932C04FB0C542705029DB0
:1002A0004FEA065847EA1637B5EB08056EEB070C20
:1002B000870E920E47EA811742EA8312A7FB0201DA
:1002C000B6EB0B0164EB00042B0D43EA0C335E1814
:1002D00044EB1C50DA465146E7FB0201C5F3130418
:1002E0004FEA0B3343EA14534FEA0432019C43EACA
:1002F0000603A4F10C040294009CCDE900B400F0C4
:100300009FF903B0BDE8F08F00200146F9E72DE921
:10031000F04D81EA030404F0004B21F0004514463F
:100320004FF0000A23F0004150EA050220D054EAC1
:1003300001021DD0C5F30A570246C5F31303C1F3EA
:100340001300C1F30A5640F4801543F48013A7EB61
:100350000608101BD64608F2FD3873EB050002D3E1
:1003600008F1010801E092185B41B8F1000F03DACF
:1003700000200146BDE8F08D00204FF480110646B4
:1003800084460EE0171B73EB050705D3121B63EBC6
:10039000050306434CEA010C49084FEA3000921865
:1003A0005B4150EA0107EDD152EA030012D082EA24
:1003B000040083EA0501084305D0101BAB4106D2B7
:1003C0000122002306E000224FF0004302E06FF01C
:1003D000010253101AEB06004CEB085110EB0A0017
:1003E00041EB0B01BDE8F04D00F01BB970B521F0F9
:1003F000004303430CD0C1F30A550024D5EB040598
:1004000064EB0403D617AD1AB34102DB00200146AA
:1004100070BD201841EB025170BDC10F80EAE07041
:100420000844CA079623002100F0CDB89623002285
:10043000114600F0C8B80EB5C10F80EAE07008445C
:10044000CA07002140F233438DE80E000A460B46EE
:1004500000F0F6F803B000BD0EB540F23341029152
:100460000021CDE900110A460B4600F0E9F803B07F
:1004700000BD00F0004220F00040C10DC0F31600A6
:1004800040F400007F2901DA00207047962903DC40
:10049000C1F19601C84001E096398840002AF4D0A5
:1004A0004042704770B5C1F30A5201F00045002484
:1004B000C1F3130140F2FF3341F480119A4201DA93
:1004C000002070BD40F233439A42A2F2334203DC73
:1004D000524200F05FF800E090402C43F1D04042DF
:1004E00070BDC1F30A5210B5C1F3130140F2FF33DE
:1004F00041F480119A4201DA002010BD40F23343EA
:100500009A42A2F2334203DC524200F043F810BD9B
:10051000904010BD2DE9F05F0546002092469B46B5
:1005200088460646814640241BE028464146474609
:10053000224600F02FF853465A46C01A914110D374
:1005400011461846224600F016F82D1A67EB0108EE
:100550004F4622460120002100F00DF817EB00095C
:100560004E41201EA4F10104DFDC484631462A46F4
:100570004346BDE8F09F202A04DB203A00FA02F14E
:10058000002070479140C2F1200320FA03F3194381
:1005900090407047202A04DB203A21FA02F0002123
:1005A000704721FA02F3D040C2F120029140084383
:1005B000194670470029A8BF7047401C490008BF72
:1005C00020F00100704710B4B0FA80FC00FA0CF083
:1005D00050EA010404BF10BC704749B1CCF12004BB
:1005E00021FA04F411FA0CF118BF01212143084348
:1005F000A3EB0C01CB1D4FEA00614FEA102042BF74
:10060000002010BC704700EBC35010440029A4BF69
:1006100010BC7047401C490008BF20F0010010BC0E
:10062000704710B5141E73F1000408DA401C41F144
:10063000000192185B411A4301D120F0010010BD66
:100640002DE9F04D92469B4611B1B1FA81F202E0DC
:10065000B0FA80F220329046FFF78DFF04460F4635
:1006600040EA0A0041EA0B0153465A46084313D0B8
:10067000114653EA010019D0C8F140025046FFF775
:1006800089FF05460E46504659464246FFF773FF1E
:10069000084305D0012004E020463946BDE8F08D2E
:1006A0000020054346EAE0762C4337430A98630569
:1006B000E40AA0EB08000022FD0A44EA47540A308D
:1006C00002D500200146E9E7010510196941DDE97D
:1006D000084500196941BDE8F04DA2E7064C074DF9
:1006E00006E0E06840F0010394E807009847103402
:1006F000AC42F6D3FFF7FEFC04B9000824B90008A9
:1007000070B58C1810F8015B15F0070301D110F8D3
:10071000013B2A1106D110F8012B03E010F8016B00
:1007200001F8016B5B1EF9D12B0705D40023521E83
:100730000DD401F8013BFAE710F8013BCB1A921CEB
:1007400003E013F8015B01F8015B521EF9D5A142E9
:10075000D8D3002070BD000070B54A4C4FF49065AE
:100760002946204600F017FA002860D02946204686
:1007700000F09EF844490888401C0880012120466A
:1007800000F0E8FA414942F21072B1F85800904284
:1007900002D2401CA1F8580009F0F0F93C4DB5F91F
:1007A0001410B5F9120007F09DFE3A4CA5F856005A
:1007B0002080A16820468847A088A5F8580004F04A
:1007C00019FF09F0DBFA344E344C307808282FD06A
:1007D00045F6AC30606042F6EF60A06042F2C400C3
:1007E000E0602F48008A2080208E6080A16B2B481B
:1007F0008847208E40F21C7180002A4C00EB81005B
:100800006887A2684FF0000550071AD5264840F2C5
:100810001A63C188491C89B2C180994207D3234B0E
:1008200049F68141198022F00401A160C58070BDA4
:1008300041F2130060604FF48060A06040F61B50EE
:10084000CEE730780A2818D2DFE800F01706130543
:100850000A050D171113EAE7BDE8704008F00EB85D
:100860000AF036FA05E0BDE8704004F04FB808F031
:1008700021FDBDE8704009F0D9BB01F0F3FD84F81B
:10088000BA5070BD00240140480700203801002004
:100890004C000020300700203F070020CC00002043
:1008A000F0010020A4020020C80A0020442C0140CE
:1008B0006FEA1121016070470029816802D041F080
:1008C000010101E021F00101816070470029816888
:1008D00002D041F4807101E021F4807181607047A1
:1008E0002DE9F041854E92B0304600F011F90BA889
:1008F00000F03FFA01214FF4C06005F079F90024BF
:100900008DF831404FF46020CDE90D044FF4A02064
:100910004FF00A080B9001278DF83C808DF830705D
:100920000BA9304600F086F9754D8DF831408DF8F1
:1009300030708DF83C700BA9284600F07BF901233C
:100940001A460F21304600F0C6F902220123114653
:10095000304600F0C0F9012303221946304600F06A
:10096000BAF9012304220021304600F0B4F9012332
:1009700005220321304600F0AEF9012306220821AA
:10098000304600F0A8F9012307220A21304600F082
:10099000A2F9012308220B21304600F09CF9012323
:1009A00009220D21304600F096F901230A22042184
:1009B000304600F090F90121304600F084F9012121
:1009C000284600F080F901231A460521304600F040
:1009D00055F901231A460621284600F04FF9002157
:1009E000304600F0CBF84FF4E041284600F0C6F85E
:1009F0000121304600F0B8F80121284600F0B4F893
:100A00000121304600F0A6F80121284600F0A2F8A6
:100A10000121304600F09EF90121284600F09AF9A4
:100A200040F61451374806F086FD12208DF840003C
:100A300002208DF841008DF842408DF8437010A8D7
:100A400004F09CFD01224FF49061304600F0E8F87C
:100A500001213046FFF73AFF01213046FFF72CFF16
:100A600001212846FFF728FF304600F06EF9304696
:100A700000F09FF80028FAD1304600F075F93046B2
:100A800000F082F80028FAD1284600F05EF92846E6
:100A900000F08FF80028FAD1284600F065F92846C2
:100AA00000F072F80028FAD10121084605F07CF820
:100AB000154D284601F050FF684601F0F0FF0F4841
:100AC00001A94C300090114881E811018020CDE946
:100AD00004404000069080000790202008904FF4CA
:100AE0004050CDE909046946284601F0BBFF0121C9
:100AF000284601F025FF12B0BDE8F0810024014036
:100B000000280140002C014008000240B4020020EF
:100B10000D4910B5884202D1012144150AE00B4964
:100B2000884202D10121041504E0094988420AD112
:100B30000121CC03204605F067F82046BDE81040AF
:100B4000002105F061B810BD0024014000280140DB
:100B5000003C01400029816802D041F4801101E08D
:100B600021F48011816070470029816802D041F42E
:100B7000004101E021F4004181607047826822F465
:100B8000E0420A43826070470146002089684907B5
:100B900000D50120704710B50246002054680B0AAA
:100BA000C9B20C401168194202D0002C00D00120BB
:100BB00010BD014600208968090700D50120704753
:100BC00038B501211C2005F013F8EF20ADF8000026
:100BD00000248DF8034003258DF8025069460D4826
:100BE00002F008FD0120ADF800008DF803408DF8FB
:100BF00002506946084802F0FDFC3B20ADF80000B9
:100C00008DF803408DF802506946044802F0F2FC6A
:100C100038BD000000080140000C014000100140F8
:100C2000002A4268C9B201D00A4300E08A43426008
:100C30007047000010B542680E4B0C791A400B68E3
:100C400042EA04221343436083680B4A1340D1E90C
:100C5000024222434C7943EA44031A438260C26A47
:100C6000097C22F47002491EC9B242EA0151C162F4
:100C700010BD0000FFFEF0FFFDF7F1FF70B5072487
:100C800009290AD9C568A1F10A0606EB4606B4404F
:100C9000A543B3401D43C56007E0056901EB41066C
:100CA000B440A543B3401D430561836BC3F30154B6
:100CB000121B921C02EB82041F22A2409343A1400C
:100CC0000B43836370BD826B491E22F4401242EADB
:100CD00001518163704770B5072409290AD9C56895
:100CE000A1F10A0606EB4606B440A543B3401D43F6
:100CF000C56007E0056901EB4106B440A543B34078
:100D00001D4305611F23072A09D2446B521E02EBC3
:100D1000820293409C4391400C43446370BD0D2A72
:100D200009D2046BD21F02EB820293409C43914094
:100D30000C43046370BDC46A0D3A02EB8202934017
:100D40009C4391400C43C46270BD816841F008012E
:100D5000816070470029816802D041F4A00101E060
:100D600021F4A00181607047816841F00401816035
:100D7000704700210160017141718160C1600121F2
:100D800001747047002800DA4042B0F5803F02DB72
:100D90004FF6FF70704780B27047000070B51E4C70
:100DA000214694F83800B1F8425006281ED9B4F80C
:100DB0004A10B4F84C00A1EB000202F10902122A19
:100DC00004D8FFF749FB0022144B0AE0884204D202
:100DD000FFF742FB0022124B03E0FFF73DFB00222E
:100DE000104BFFF722FAFFF77CFB09E005D12846FC
:100DF000FFF732FB0C4A0D4BF3E70D4951F8200089
:100E0000C5EB45116063B0EB410F03D9C5EB45104D
:100E10004000606370BD00005804002000003440B2
:100E200000003340000035406766666666E64B406A
:100E300088AF000810B50C4C2078400713D5FFF799
:100E4000ADFF0A49A08E088008483038018821F09B
:100E500010010180001F018841F0100101802078FD
:100E600020F00400207010BD580400204004004011
:100E7000F0B4254B002103F134009A793AB1234AAA
:100E800041F2CD05B2F90240AC4211DC99711E4C21
:100E900082683434C2F3C006C2F300252468AE422F
:100EA00011D1240706D5D40506D442F0080205E086
:100EB0009180C162F0BC704722F008028260998282
:100EC000012098711AE090F84A60D6B9104E766CFD
:100ED000B6F5966F15DC240713D49C8AB4F5FA6F27
:100EE00002D2641C9C82E5E70A4B65F3C3021C78BE
:100EF00024F001041C70598019828260F0BC07F054
:100F0000DDBF9982D6E7000070020020E2050020D4
:100F100038010020B00A0020012180F82E104FF483
:100F2000AF6101861F21418645F27151818670476C
:100F300070B506464089204B204C4FF400510025E7
:100F400080B362887AB1012A0CD1E188491C89B248
:100F5000E1803289914205D36580E580FF2801D088
:100F6000401E708170BD70882288904201D9012294
:100F700000E00022184602F0C6FB7088B1880144E8
:100F80002088401C80B220808142EBD82580A08838
:100F9000401C80B2A080F1888842E3D301206080A9
:100FA000A58070BDFFE70022184602F0ACFBA580CB
:100FB000E58025806580F4E700100140C805002029
:100FC000FEE7000010B5074C0021204600F0AEF807
:100FD0000121204600F0AAF82046BDE81040022179
:100FE00000F0A4B80064004010B50D4C0B49204639
:100FF00000F0AEF809492046891C00F0A9F809491B
:10100000204600F0A5F8084C206807F057FC0021A6
:1010100006A008F0B1FC206010BD00000200F01036
:10102000006400407000F0304C0800206465765F7A
:1010300063616E31000000001E491F480A78FF2AD4
:1010400004D002704A78FF2A02D106E05422F8E761
:1010500042708A78FF2A02D106E05122F8E78270B6
:10106000CA78FF2A02D106E00522F8E7C2700A79A1
:10107000FF2A02D106E04022F8E702714A79FF2AEE
:1010800002D111E06022F8E74271887901220B4910
:10109000FF280BD050B1012808D0022801D0032826
:1010A00001D181F84A0070475922EDE781F84A20C2
:1010B0007047000000E40108A7070020A4020020F8
:1010C00070B51848017861F30704417861F30F2483
:1010D000817861F31744C17861F31F640179407925
:1010E00061F3070560F30F2502F08CF80E4E3046D1
:1010F00002F030F8A1B2304602F068F8210CB01CC2
:1011000002F064F8A9B2301D02F060F805482838F2
:10111000C07800F00301B01D02F058F8BDE870403F
:1011200002F04CB8A707002000E4010841B10129F2
:101130000AD0022903D1816841F40001816070471F
:10114000816841F08001F9E7816841F40041F5E7E9
:101150000A4A914202D1002181617047C1F3130212
:101160008B0101D5C26070474B0101D50261704708
:10117000090101D582607047426070477000F0300D
:1011800030B5082310240422B1F5007F1DD010DCF7
:10119000202929D007DC012921D0042922D00829BF
:1011A00000D1C46030BD402920D0B1F5807FF9D195
:1011B0000BE00025B1F5004F06D008DCB1F5806FDB
:1011C00003D0B1F5006FEDD18561426030BDB1F55E
:1011D000803F0DD0B1F5003FF8D1446030BD0549E6
:1011E000816030BDC36030BD036130BD046130BD7E
:1011F000436030BD010101003EB5684600F026FAAB
:1012000000208DF8080001218DF809108DF80A00E2
:101210008DF80B108DF806001D498DF807008DF82C
:10122000020001F11000897C8DF80310C1788DF85F
:10123000041001798DF80510C088164CADF8000037
:101240006946204600F045F901220221204600F0BF
:1012500038F901221146204600F033F90E492046A4
:10126000FFF776FF0C492046891CFFF771FF0B49F9
:101270002046FFF76DFF08492046491EFFF768FF2B
:1012800001224FF40441204600F01BF900203EBD2E
:101290005C080020006400400200F0107000F03094
:1012A000094910B588424FF0010101D14C0601E017
:1012B0004FF08064204604F08FFC2046BDE81040CB
:1012C000002104F089BC0000006400402DE9FF47C4
:1012D0000026012119488DF80B608DF80C10DFF8FD
:1012E0006090ADF808608DF80D10354634464FF02B
:1012F000040809F1800AC7681AE000BF8DF80A40A7
:1013000059F82610761C480BADF8000008EBC10117
:10131000ADF802105AF825106D1C4A0BADF80420E8
:1013200008EBC100ADF80600684600F00BF8641C3D
:10133000BC42E3DB04B00020BDE8F0874808002091
:10134000B0180020F0B5827A012191402E4A13682E
:1013500043F0010313602C4B1C331C688C431C604E
:10136000294D067B294C0C35A6B92E688E432E607C
:101370004688C78846EA0746877A04EBC707C7F856
:1013800040660688878846EA0746877A04EBC707DF
:10139000C7F84466067B012E12D12E680E432E60DC
:1013A000867A056804EBC6064FEA3545C6F840560E
:1013B000867A456804EBC6044FEA3545C4F84456BE
:1013C000114CC57A241D002D256806D00D432560DB
:1013D0000D4C0589143415B104E08D43F7E72568F9
:1013E0008D4325600589012D02D125680D432560B7
:1013F000407B012802D1186808431860106820F06B
:1014000001001060F0BD0000006600400060004078
:101410000246002053690B424AD0B1F5807F3BD091
:1014200013DC08292ED007DC012926D0022927D079
:1014300004293DD1D0682BE0102925D0202926D0C1
:10144000402935D11069102130E0B1F5004F2BD083
:101450000BDCB1F5007F22D0B1F5806F22D0B1F561
:10146000006F25D19069702120E0B1F5803F11D047
:10147000B1F5003F1CD15068E5E790680D4915E0D3
:10148000D06802E0D068DEE7106903210EE0106941
:1014900008210BE05068FBE79069012106E09069A4
:1014A000022103E0906900E05068042100F0B4BF1D
:1014B00070470000010101008069C0F302100001C3
:1014C0007047002A426901D00A4300E08A43426122
:1014D000704710B50368002223F00203036003681D
:1014E00043F0010303604FF6FF7300E0521C4468B1
:1014F000E40701D19A42F9D14268D2073ED08A79F5
:10150000012A02683CD022F080020260CA79012AD6
:10151000026838D022F0400202600A7A012A02688A
:1015200034D022F0200202604A7A012A026830D0C8
:1015300022F0100202608A7A012A02682CD022F07E
:1015400008020260CA7A012A026828D022F0040246
:1015500002608A78CC78920742EA04620C7942EA07
:1015600004424C79098842EA0452491E0A43C26186
:10157000016821F001010160002114E0002010BD8C
:1015800042F08002C1E742F04002C5E742F020028B
:10159000C9E742F01002CDE742F00802D1E742F07D
:1015A0000402D5E7491C4268D20701D09942F9D11B
:1015B0004068C007E2D1012010BD000010B500EB6B
:1015C0000113D3F8B04114F004041472D3F8B041FD
:1015D00034D0E408C2F80440D3F8B04104F0020467
:1015E0005472D3F8B44104F00F049472D3F8B441A8
:1015F000240AD474D3F8B841D472D3F8B841240A79
:101600001473D3F8B841240C5473D3F8B841240EA2
:101610009473D3F8BC41D473D3F8BC41240A147436
:10162000D3F8BC41240C5474D3F8BC311B0E937412
:1016300039B1016941F02001016110BD640D1460F0
:10164000CAE7C16841F02001C16010BD002181716D
:10165000C171017241728172C1728170C1700321C6
:1016600001710221417101210180704730B50246AC
:10167000002093685B0108D49068000101D5012027
:1016800003E09068C00037D5022002EB0012D2F8C8
:10169000803103F00103C2F880310B7A73B3D2F8C2
:1016A00080414D681C434B7A43EAC5031C43C2F892
:1016B00080418B7A03F00F038B72D2F8843123F0D0
:1016C0000F03C2F88431D2F884318C7A2343C2F8F4
:1016D0008431CB7ACC6843EA0423C2F88831CB7BCF
:1016E000096943EA0121C2F88C11D2F8801141F056
:1016F0000101C2F8801130BD042030BDD2F8803124
:101700004C7A23430C8843EA4453C2F88031D0E733
:101710002DE9F04FFE488BB0DFF8FC93416C1A20A6
:10172000B1FBF0F084B20D20B4FBF0F00290F94868
:101730004D46B0F91A00C0F30F100490B9F910002B
:1017400001F080F842F210710844FEF785FEF34A7A
:10175000F34BFEF76AFDFEF7C4FE80B20990B5F9BF
:101760001E0001F06FF80890B5F9200001F06AF84A
:101770000790B5F9220001F065F8EA4B0690D88B86
:101780004FF4FA71484340F6FF71B0FBF1F0DFF817
:1017900098C385B2E54EBCF81000E5490590F08885
:1017A0000A78070967F30002C70A67F34102C7080E
:1017B00067F38202870867F3C302070B67F304121B
:1017C000470867F3451260F38612470B67F3C712A9
:1017D0000A704A78470A67F30002470967F3410233
:1017E000870967F38202070A67F3C302C70967F331
:1017F0000412377ABF0867F34512800B60F3861234
:101800004A7093F8070110B142F0800001E022F025
:1018100080004870B27A88789B4662F341001A468D
:101820001B89B246DE0886EA1326F64366F3820079
:101830009CF8006066F304105E0966F34510DB0A4D
:1018400063F386101388DB135B1C63F3C710887087
:101850009BF84A202AB1012A07D0022A0AD0032A7B
:101860000DD0CA7822F003020CE0CA7822F00302FD
:10187000521C07E0CA7822F00302921C02E0CA78E8
:1018800042F00302AA4BCA702833A3F118069A78D3
:1018900002F00302012AB27811D022F01002B270D5
:1018A000CA7897070ED020F00800887058799846BB
:1018B00000F00300012808D0022809D00BE042F014
:1018C0001002ECE740F00800EFE742F0040001E00E
:1018D00022F00400C870964F2246791DF87820F057
:1018E0009000F870381D04F0E1FF924CB4F902004A
:1018F00005F08FFEB871B4F9040005F08AFEF871A6
:1019000007F10804611C2046049A04F0CFFFE11C93
:10191000A01C099A04F0CAFF87486421B0F90400AA
:101920004843800B03F042F960712A46E11DA01D77
:1019300004F0BCFFB9F91000FFF724FAC8214843AE
:10194000800B03F033F9307098F80000474601230C
:101950004FF00208B3EB901F03D1B07840F00100C4
:1019600005E0B8EB901F03D1B07820F00100B07013
:10197000797801F00300012802D0022804D007E0A2
:10198000B07840F0020002E0B07820F00200B070C1
:10199000DBF80820B078D50965F38200B070BD7817
:1019A0005C46C5F38105012D02D0022D03D005E070
:1019B00040F0200001E020F02000B0709B46B3EB27
:1019C000911F03D1B07840F0800005E0B8EB911F83
:1019D00003D1B07820F08000B07058483146B1464D
:1019E000437FF07863F34100D30A63F3820094F8F5
:1019F0002A3163F30000237963F3C300F0709AF88F
:101A00000A503079534665F3820025786D116D1CBC
:101A100065F3C300550965F30410087110164A797F
:101A2000401C60F3C3024A719AF80020C879404D07
:101A300062F30300DA881835D20B62F386109AF845
:101A40000820691CD20862F3C71089F807002846ED
:101A5000029A04F02BFFE91CA81C059A04F026FF4B
:101A6000B4F9E800FFF78EF9C8214843800B03F072
:101A70009DF82871207AC109A87961F3C710B4F8DC
:101A8000C8100A0A62F30600A871E971273D691CB3
:101A90002846089A04F00AFFE91CA81C079A04F0DB
:101AA00005FF691D281D069A04F000FF0298A87121
:101AB000103D287800287DD0E07B00287AD128705E
:101AC00005F11700017801F00301012904D0017824
:101AD00001F00301022904D10278397862F301018F
:101AE00039700178C1F38101012904D00178C1F373
:101AF0008101022905D101788A08397862F38301CE
:101B000039700178C1F3011101291DD0017817E066
:101B100038010020D0040020380500209A999999B6
:101B20009999B93FA4020020B00A0020000C0020BF
:101B30007F070020F80D0020E2050020200E002085
:101B4000C1F30111022905D101780A09397862F33C
:101B50000511397002785946BBEB921F03D0027809
:101B6000B8EB921F05D1027813093A7863F3871214
:101B70003A70427802F00302012A04D0427802F05F
:101B80000302022A04D142787B7862F301037B705E
:101B90004278C2F38102012A04D04278C2F3810262
:101BA000022A05D1427893087A7863F383027A7027
:101BB000427800E02CE1C2F30112012A04D04278FD
:101BC000C2F30112022A05D1427813097A7863F32D
:101BD00005127A704278B1EB921F03D04278B8EBCD
:101BE000921F05D1427813097A7863F387127A70CD
:101BF000827802F00302012A04D0827802F0030204
:101C0000022A04D18378BA7863F30102BA70827829
:101C1000C2F38102012A04D08278C2F38102022A2F
:101C200005D182789308BA7863F38302BA70827818
:101C3000C2F30112012A04D08278C2F30112022AEF
:101C400005D182781309BA7863F30412BA708278E6
:101C5000B1EB921F03D08278B8EB921F06D1827845
:101C6000C2F30113BA7863F34712BA70C278D2068E
:101C700009D0C27802F01F021F2A04D2C278FB7872
:101C800062F30403FB70C278520905D0C27853098D
:101C9000FA7863F34712FA70027902F00302012A1C
:101CA00004D0027902F00302022A04D102793B79BE
:101CB00062F301033B710279C2F38102012A04D06D
:101CC0000279C2F38102022A05D1027993083A7996
:101CD00063F383023A710279C2F30112012A04D03C
:101CE0000279C2F30112022A05D1027913093A7965
:101CF00063F305123A710279B1EB921F03D00279B6
:101D0000B8EB921F05D1027913093A7963F3871270
:101D10003A71427902F00302012A04D0427902F0BA
:101D20000302022A04D142797B7962F301037B71B9
:101D30004279C2F38102012A04D04279C2F38102BE
:101D4000022A05D1427993087A7963F383027A7182
:101D50004279C2F30112012A04D04279C2F301127E
:101D6000022A05D1427913097A7963F305127A714F
:101D70004279B1EB921F03D04279B8EB921F05D1A3
:101D8000427913097A7963F387127A71827902F0C2
:101D90000302012A04D0827902F00302022A04D14C
:101DA0008279BB7962F30103BB718279C2F381024C
:101DB000012A04D08279C2F38102022A05D18279F4
:101DC0009308BA7963F38302BA718279C2F301127C
:101DD000012A04D08279C2F30112022A05D1827944
:101DE0001309BA7963F30512BA718279BBEB921FBA
:101DF00003D08179B8EB911F05D181790A09B979AE
:101E000062F38711B971C179F87961F30300F87150
:101E1000434E307800F00F00042801D1FFF750F94D
:101E20003878C0F3810001283AD1F079010637D51E
:101E300000F07F00142833D899F8021041F0040113
:101E400089F80210374AC9B28B07107F4F464FF40A
:101E50007F412AD580281FD3334B00F01F00126822
:101E600053F82000024217D1A06840F08070A060B3
:101E70002B4830388078C0071BD0A068C00118D527
:101E80002A48406C322814D868888846404527D1B3
:101E900001F056FC68800DE0A06820F08070E6E755
:101EA00099F8021021F00401CAE7A06820F08070C0
:101EB000A0606980B878800702D40020AAF80A00E0
:101EC0003079C00701D0AAF80AB09AF80A00C10711
:101ED0001348A0F14900017812D041F0010111E04E
:101EE00001F016FC40F6B8318842E3D3A068C10186
:101EF000E0D50005DED4AAF80AB0A5F80280D9E73B
:101F000021F001010170A168C901017802D541F0F9
:101F1000020101E021F0020101700BB0BDE8F08F79
:101F2000AF070020E8050020E8B3000838010020D2
:101F300070B51548006810F0E05F23D0134CD4E969
:101F4000001081421ED004EB001104F5A1608A68E4
:101F500042600A7B827204230372002545720B30B3
:101F60000E31FEF710F972B66068401C60604028C0
:101F700000D3656062B60649BDE870400248083883
:101F8000FFF774BB70BD000008640040A814002077
:101F9000B0190020FCB505464FF6FF7600200C4630
:101FA000ADF8006048F205078DF8040020E000BF9E
:101FB00015F8010B8DF8040001A9084602F082FB18
:101FC000BDF800009DF8041080EA0120ADF8000083
:101FD0005FF00000BDF800100A0402D587EA410155
:101FE00001E006EA4101401CADF800100828F1DBD1
:101FF000641EDDD26946084602F04EFBBDF80000C3
:10200000FCBD00000246002004E000BF12F8013BC6
:102010001844C0B2491EF9D27047000070B5144A86
:1020200085B010880024134901940094039420463D
:102030000494138807E0CD8B009E354400950D8BEA
:10204000019E3544019515889D42F4D0401CC0B2D4
:102050008028EED300984111074841808480019880
:102060004111064881830183818205B070BD000063
:1020700048070020A4020020E2050020D004002030
:1020800030B4104C002003464FF47F42A4F13401D9
:1020900021F8103024F81020401C1A28F8DB0A4BD5
:1020A000002000BF33F8104021F81040401C1A28CF
:1020B000F8DB064806490280012081F8300030BC78
:1020C00003F052B96C100020080800203C080020E2
:1020D000CC0E00202DE9F84303F092F9C64DC54B14
:1020E00000204FF47F4105F1340400BF35F8106043
:1020F00033F81020964203D025F8102024F8101051
:10210000401C1A28F2DBBD4890F83000012808D0A6
:102110005FF0000024F81010401C1A28FADBBDE81C
:10212000F88302F0F3FD208801F0F2FA2988B44E1A
:1021300088420AD301F004FB2080B24800906B462D
:102140000822B149306808F085FE608801F0E0FAA5
:10215000698888420CD301F0F3FA6080A948AA4943
:10216000401C00906B4608220831306808F072FE6F
:10217000A08801F0CDFAA98888420CD301F0E0FADA
:10218000A080A048A049801C00906B460822103116
:10219000306808F05FFEE08801F0BAFAE98888420A
:1021A0000CD301F0CDFAE08096489749C01C00900E
:1021B0006B4608221831306808F04CFE208901F087
:1021C000A7FA298988420CD301F0BAFA20818D48F8
:1021D0008D49001D00906B4608222031306808F0C0
:1021E00039FE608901F094FA698988420CD301F0C4
:1021F000A7FA608183488449401D00906B460822FD
:102200002831306808F026FEA08901F081FAA8463E
:10221000A98905277D4D884216D36878052813D2F1
:1022200001F08EFAA0816878401CC0B26870052861
:1022300000D96F7073487449303000906B460822A3
:102240003031306808F006FEE08901F061FAB8F834
:102250000E10884216D3A878052813D201F070FA20
:10226000E081A878401CC0B2A870052800D9AF70E2
:1022700064486549313000906B4608223831306837
:1022800008F0E8FD208A01F043FAB8F810108842FF
:1022900016D3E878052813D201F052FA2082E878A4
:1022A000401CC0B2E870052800D9EF705548564967
:1022B000323000906B4608224031306808F0CAFD89
:1022C000608A01F025FAB8F81210884216D32879EE
:1022D000052813D201F034FA60822879401CC0B27C
:1022E0002871052800D92F7146484749333000909E
:1022F0006B4608224831306808F0ACFD208D01F0B3
:1023000007FAB8F82810474688420BD301F018FAAC
:1023100020853F483C4900906B460822A031306838
:1023200008F098FD608D01F0F3F9798D88420CD3A7
:1023300001F006FA608536483349401C00906B4630
:102340000822A831306808F085FDA08D01F0E0F981
:10235000B98D88420CD301F0F3F9A08529482A49A8
:10236000503000906B460822B031306808F072FDA2
:10237000E08D01F0CDF9F98D88420CD301F0E0F940
:10238000E08520482049603000906B460822B83133
:10239000306808F05FFD208E01F0BAF9398E88426E
:1023A0000CD301F0CDF92086164817496130009012
:1023B0006B460822C031306808F04CFD608E01F099
:1023C000A7F9798E88420CD301F0BAF960860D48DE
:1023D0000D49623000906B460822C831306808F021
:1023E00039FD0C48FFF768F800283FF498AE2870D4
:1023F00095E600000808002038100020CC0E0020D0
:102400004C0800200002FF18000F002040080020A8
:102410000006FF1800640040024600200A4200D077
:102420000120704730B50E4902880A800C4A438863
:10243000083A13800B1F808818802024151F2C80D9
:102440000020401C80B23C28FBD341F69910088044
:1024500044F64800108046F6480018802C8030BDB5
:10246000202C0140114944F648000880091D46F619
:1024700048000880091D41F6991008800B48001F8C
:10248000018841F02001018009480021A0F868106E
:10249000A0F86610A0F86410A0F86210A0F8601010
:1024A000A0F85E100348418181827047182C0140DA
:1024B000A40200204C0000202DE9F04F4B4B4C486B
:1024C0000021DA7A0678802A26F001057AD31C6882
:1024D000484B02F01F0253F82220474B14421A685F
:1024E00002D042F0200201E022F020029946DFF8FB
:1024F0000CB11A60434B404F9BF80040DFF800A13D
:10250000B3F9043097F84AC0022C5CD1D9F80870AE
:10251000C7F3C004C7F30028444554D0364C343CBC
:1025200094F80280B8F1000F06D0B8F1010F0DD079
:10253000B8F1020F4CD120E0110549D5910647D4DE
:102540000121A17026F00401017041E015053FD47E
:1025500095063DD575073BD4458895BB4380002B38
:1025600009DD46F0050101700221A1702649B1F88C
:10257000441001822CE0A1702AE0C6880EB9002B1D
:1025800014DC067B664511D1204EB6895FEA467899
:102590000CD45FEA867809D45FEA427806D55FEA10
:1025A000826803D5F60701D1FE0111D5057041807F
:1025B000AAF8001041810182A17089F80F108BF8F0
:1025C000001005E00EE005704180AAF8001041817E
:1025D000C38080F80CC0500960F3CB22C9F80020FA
:1025E000BDE8F08F057041804181F9E7E8050020E2
:1025F000B00A0020E8B30008A40200203F07002032
:102600000C010020E205002038010020000C002011
:102610002DE9F04796B000240C940D940E940F947D
:1026200072B68048816941F400718161816941F429
:10263000806181614FF4004003F0ACFA7A4D0021D3
:102640002846FEF743F900212846FEF735F9774E74
:1026500000213046FEF730F9754F0021384600F072
:102660006FF901204FF47041401C8842FCD328468A
:10267000FEF74EFAB1463046FEF74AFA384600F009
:102680006BF94FF46020CDE912048DF8454001202C
:102690004FF004088DF8440010948DF8508010A974
:1026A0002846FEF7C7FA01231A4605212846FEF7F9
:1026B00012FB0123022206212846FEF70CFB012310
:1026C000032207212846FEF706FB012304220F21DF
:1026D0002846FEF700FB384600F03EF9684600F059
:1026E000DEF95148534E4C300090CDF80C80CDE9C6
:1026F00001648020CDE904404000069080000790EE
:10270000202008904FF44050CDE90904694638462E
:1027100000F0A8F901212846FEF7D8F80121384633
:1027200000F00EF901212846FEF7C6F847F23050B6
:1027300015941599491C15918142FAD30121284617
:10274000FEF708FBADF82C40A04640F2DC5A4FF4EF
:10275000007420E05046CDF854801599491C15911D
:102760008142FAD330880D9908440D9070880E99F3
:1027700008440E90B0880F9908440F90F0880C9987
:1027800008440C9001212846FEF7E4FABDF82C001D
:10279000401CADF82C00BDF82C00A042DAD30D98F7
:1027A000C11124480A3001830E99C91141830F9940
:1027B000C91181830C99C91181801F49C9884904B5
:1027C00007D41E49028B21F85C2F428B4A80808BF4
:1027D000888000212846FEF779F80021384600F06D
:1027E000AFF800212846FEF767F800214C4648461E
:1027F000FEF762F80220C102401C8842FCD3284642
:10280000FEF786F92046FEF783F9384600F0A4F873
:10281000FEF766F80A493C20087062B616B0BDE8BB
:10282000F087000000100240002401400028014011
:10283000080002402E050020000C0020580E002049
:102840003C07002010B5FEF79DFA4FF42F61484376
:10285000800B10BD70B5204B40F6C81441F2B7058F
:102860005B6C48F6E6065C4305EBA4341B4D7343F2
:102870004EF6F61606EBA333C5E90443D460401ABE
:10288000536110609168884202DA4942884200DC54
:10289000116010684343107E0341906A19189162D9
:1028A000506A814200DD9062916A106A814201DBC8
:1028B000084600E09062A86111684C43117C0C410D
:1028C00008412118B2F91C00884204DBB2F91A0051
:1028D000884200DC08B270BD3801002014010020DD
:1028E00010B54FF40054204600F0ACF8002813D087
:1028F0000A49087840F008000870204600F014F8F3
:102900000021074800F01CF80648C17E012903D1C8
:102910000021C1760121017710BD00008206002050
:1029200044000240040D0020C10002D502490860A5
:1029300070470249486070470404024000000240AA
:102940000029016802D041F0010102E04FF6FE7259
:10295000114001607047000001684FF6FE7211409F
:1029600001600021016041608160C1603149314AEC
:102970000839904203D1486840F00F0006E02D4A24
:102980001432904204D1486840F0F000486070472B
:10299000284A2832904203D1486840F47060F5E735
:1029A000244A3C32904203D1486840F47040EDE73D
:1029B000204A5032904203D1486840F47020E5E745
:1029C0001C4A6432904203D1486840F47000DDE74D
:1029D000184A7832904203D1486840F07060D5E7D9
:1029E000154A111F904203D1086840F00F0006E01D
:1029F000114A1432904204D1086840F0F000086097
:102A000070470D4A2832904203D1086840F4706044
:102A1000F5E7094A3C32904203D1086840F470401F
:102A2000EDE7054A50329042EAD1086840F4702040
:102A3000E5E700000800024008040240406880B258
:102A40007047000001460020CA0001D5034A00E09B
:102A5000034A12680A4200D0012070470004024075
:102A60000000024030B5036847F6F07293430C6AE9
:102A70008A682243D1E904452C4322438C692243CE
:102A8000CC6922434C6A22438C6A22431A43026077
:102A9000CA6842600A6882604968C16030BD00212E
:102AA000016041608160C160016141618161C1611A
:102AB000016241628162704710B5114C8CB00021F7
:102AC0002046FFF73DFF2046FFF746FF0D480090E8
:102AD0000D480021CDE901016420CDE903018020EA
:102AE000CDE905010791089109910A9169462046AF
:102AF000FFF7B8FF01212046FFF722FF0CB010BD01
:102B00005800024004380140F0080020F0B540F6BB
:102B1000AA222A49C284838B0C88E31A9BB20F2B0A
:102B20000DD309888183037E00213BB1244BB3F987
:102B30000A40244B062C03DA818429E08184F0BD0D
:102B4000214C2478022C02D0002CF5D0F0BD1F4C73
:102B500040F68B27656C1B4CA5F22D16BE42B4F9CE
:102B6000004017D2418B491C89B241836429EDD3BF
:102B700064214183B0F92410914201DA01EB221261
:102B80008284641C20B24FF4007118808842DDDB1F
:102B90001980F0BD41F29416B542FADBB0F9245029
:102BA000002D02DDA5EB221200E000228284418389
:102BB000641E20B218800028EADDF0BD480700201E
:102BC0004C000020540400203F0700203801002062
:102BD00010B50446B0F9020043F699114843811339
:102BE000E06840F26662504301EBA030E060B4F967
:102BF000001043F6991251438A13216940F266632B
:102C0000594302EBA131216105F00CFC6061A18800
:102C100040F6AB2208444010A0F515415539E0625A
:102C2000914205D9A0F5F851FF39521C91421DD2AD
:102C300049F25451884202DDA0F5204002E0A0F59F
:102C4000F850FF38206300EB400040F34F00208530
:102C5000B4F924104A42904201DA104602E0884258
:102C600000DD0846E083228461848AE0A0F5FE420C
:102C7000FF3A41F255518A4214D8A2F6AA202063A5
:102C800000EB400040F34F002085B4F9242051426E
:102C9000E183884201DA084602E0904200DD1046F6
:102CA000404250E0A0F5D442AA3A8A4215D2A2F698
:102CB000AA20206300EB400040F34F012185B4F9C6
:102CC00024004242E2832084914201DA104602E06D
:102CD000814200DC0846608453E0A0F5AA42543AE1
:102CE00041F256539A4215D2A2F6AB20206300EB74
:102CF000400040F34F002085B4F924104A4290422E
:102D000001DA104602E0884200DD08464042E083D6
:102D1000218419E0A0F5804241F254539A4215D221
:102D2000A2F6AA20206300EB400040F34F0020856C
:102D3000B4F92410E1834A42904201DA104602E0DD
:102D4000884200DD0846208462841AE0A0F52852FB
:102D5000AB3A8A4215D2A2F6AA20206300EB4000CB
:102D600040F34F012185B4F92400E08342422284DC
:102D7000914201DA104602E0814200DC08464042FE
:102D8000A9E7B4F91E0041420948B0F900004143E7
:102D90008913E180B4F9201049424143891321810C
:102DA000B4F92210494241438813608110BD0000EC
:102DB0005404002000210176704770471548164AD8
:102DC0004FF480410078042821D002F13C03D08ADE
:102DD0009B88C01A00B22F2801DD001108E00028EE
:102DE00001DD002007E00D4B984201DA184602E0B1
:102DF000402800DD40209389184400B2884203DC5B
:102E000040F26661884200DA0846908170479181FD
:102E1000704700003F070020D0040020C0FEFFFFE5
:102E200038B54B484B4902880B889A1A92B20F2A40
:102E300071D30988484C01804FF0FF01E2884FF4BC
:102E40007A7355044FF4967002D51622009103E070
:102E5000950403D515220091014670E0D50402D5F2
:102E600014220091F8E7150502D513220091F3E72B
:102E7000550502D512220091EEE7950502D51122E3
:102E80000091E9E7D50502D510220091E4E7150687
:102E900002D50F220091DFE7550602D50E220091E0
:102EA000DAE7950602D50D220091D5E7D50602D5C1
:102EB0000C220091D0E7150702D50B220091CBE739
:102EC000550702D50A220091C6E7950702D50922C7
:102ED0000091C1E7D20702D008220091BCE7228905
:102EE000550702D507220091B6E7950702D50622BD
:102EF0000091B1E7D20702D005220091ACE7A27A97
:102F0000D20702D004220091A6E7A289D40603D5F5
:102F100003220091A0E719E0140702D502220091D4
:102F20009AE7540703D4940701D4D20702D00122B0
:102F3000009191E70020034602460146009003F00D
:102F4000D1FBBDE838400248FDF7F2BF38BD0000B4
:102F5000F40B002048070020000C0020F0B5594871
:102F6000594982880B889A1A92B29C2A64D309889C
:102F7000818056490A880146002A0B7843F00201F5
:102F800056D11646524A1C0715680246127822F09E
:102F9000020274D54F4C0746E4887F785FEA845C70
:102FA00002D547F0010701E027F001074770A704A9
:102FB000477802D547F0020701E027F00207477083
:102FC000670401D4E70703D0477847F00807477044
:102FD000640603D5447844F0040404E01C0603D4DA
:102FE000447824F004044470EC0450D4354C9A071F
:102FF000247824F0100423D4324D42782F7A2D788F
:10300000012A45F0100514D0022A16D02D4C042AAE
:10301000A47804F1010C0CF0FF0C13D0072A25D082
:10302000032A23D0052A21D0062A1FD021F010011F
:1030300042E0B90702E00570F0BD39070029FADB6C
:103040000470F0BDFA0601D41A060AD50170022CEC
:1030500004D280F802C0BCF1020FF2D341F080012B
:103060002AE021F0100101708670F0BD877A7F069A
:10307000F7D5032C04D8017080F802C0F0BD0FE032
:103080005107D8D51906D6D443F0800114E0027058
:103090004178CB0701D18907F0D522F010010BE070
:1030A000E9040BD49907E9D4818AC82902D2491CC2
:1030B0008182E3E743F00A010170DFE70270868254
:1030C000DCE7000010070020480700204A07002026
:1030D000A4020020000C002070B51148114C4FF0E4
:1030E0000005C088810503D4410601D4C00515D56B
:1030F0004FF480610C4800F0FBFA68B9A08840F6F4
:10310000B831884201D2401CA08080B2B0F57A7FED
:1031100001D30120607070BDA58070BD6570FBE7B4
:10312000000C002060070020000C0140084946F612
:1031300068000880091D0880091D41F6DD500880DF
:103140000348001F018841F0200101807047000002
:10315000182C014070B50D4E0546304600F05EF863
:10316000042811D10A4C206940F0020020616561F9
:10317000206940F040002061304600F04FF821699E
:1031800041F6FD721140216170BD0000FFFF0F008C
:103190000020024008490420CA68D20701D001205B
:1031A0007047CA68520701D502207047C968C9062E
:1031B000FBD503207047000000200240024801694F
:1031C00041F080010161704700200240F0B50646E1
:1031D0004FF6FF770D46384600F020F804280DD151
:1031E000074C206940F0010020613580384600F02E
:1031F00015F8216941F6FE7211402161F0BD000011
:103200000020024003480249416003494160704781
:103210002301674500200240AB89EFCD00B503468E
:10322000FFF7B8FF03E000BFFFF7B4FF5B1E012804
:1032300003D0002B00D1052000BD002BF4D1FAE70C
:1032400010B5C28800210AB1032206E002890AB142
:10325000022202E0428912B10122027000E00170F4
:1032600004784FF4804344F6206244B1012C06D028
:10327000022C07D0032C01D14180818010BD4380F6
:10328000828010BD41F23331418040F6B731F4E71E
:10329000401A10609168884202DA4942884200DC94
:1032A000116051691068137E41431941936A0B44C0
:1032B0009362516A8B4200DD9162936A116A8B427C
:1032C00000DA9162D168936A4143107C0141034165
:1032D000B2F91C001944884204DBB2F91A00884292
:1032E00000DC08B270470000054920B1086940F0D1
:1032F0008000086170470348486003484860704791
:103300000020024023016745AB89EFCD06494FF409
:103310007A70CA68D20705D0401E0004000CF8D1AC
:10332000FF20704700207047002002400E4A032013
:10333000A2F14C0182F83E000020C8800B490886AB
:10334000C862C8830884488490620948016DB1F559
:10335000206F01DBA3219162807A002802D0906A5D
:1033600040429062704700004C0000203805002069
:1033700038010020F0B53D4988894A89801A80B219
:103380000F286AD388894881CA8939480B3A272A85
:1033900026D28A7822BB8268384B42F480728260DF
:1033A000344A374C374D12785607334A0AD4364ED2
:1033B00036881680354A12881A80354A128822804B
:1033C000344A09E0344E36881680344A12881A800E
:1033D000334A12882280334A12882A8001228A7056
:1033E000314A0021314B82F84D1019469A7F304DF9
:1033F0000968802A32D302F01F0255F822201142B8
:103400002CD0826822F48012184E82601236144644
:103410001215B778521C62F38617264AB77093F8D4
:1034200016C01778BCF1800F27F0020608D30CF005
:103430001F0C55F82CC011EA0C0F01D147F0020601
:1034400016701A7E802A0DD302F01F0255F8222032
:10345000114207D144F400218160F0BD826842F43A
:103460008012D1E724F40021F6E700003C07002099
:10347000A402002038010020C8040020CA04002053
:10348000CC040020CE040020B8040020BA040020A0
:10349000BC040020BE040020C0040020C2040020A0
:1034A000C4040020C6040020580E0020E8050020B7
:1034B000E8B30008D004002070B521488189028952
:1034C000891A89B20F2932D381891E4D1E4C018180
:1034D000697A22681D4E42F00400802908D301F069
:1034E0001F012B6856F821100B4201D122F0040075
:1034F0002060FFF7F1FDA87B802819D300F01F00A2
:10350000296856F82000014212D1206820F00200FC
:103510002060E87A80280FD300F01F00296856F851
:103520002000014208D1206820F00800206070BD12
:10353000206840F00200EBE7206840F00800F5E763
:103540003C070020E8050020A4020020E8B30008A2
:1035500030B5044600204FF40043024640EA030120
:1035600001FB01F5A54200D80846521C5B0812B2C7
:10357000102AF3DB30BD0000F0B51D4C1B4A4FF0A4
:10358000010C94F83B5094F80AE0144692F83C3051
:1035900094F838402B43651CEEB2154D95F83D70FC
:1035A0000025BEF1FF0F0AD0BEF1000F06D18B42FD
:1035B00013D155700C2C01D282F83860F0BD8342D3
:1035C00002D182F801C0F5E78B42F7D15570B807F8
:1035D00009E000BF82F83850F0BD8342FCD1F843C7
:1035E00082F801C080070028F4D0F0BD5804002004
:1035F00038010020F0B5CA78002502F00F03D2068A
:1036000001D58A7813430A784FF00F0E12F0FF0F9E
:103610004FF001021CD004680F8802FA05F637400B
:10362000B74211D14FEA850C0EFA0CF724EA0707CE
:1036300003FA0CF43C43CF78282F02D0482F02D055
:1036400002E0466100E006616D1C082DE4D30460D1
:103650000C88FF2C1ED944685FF0000606F10807AD
:1036600002FA07F50F882F40AF420FD14FEA860CC0
:103670000EFA0CF7BC4303FA0CF73C43CF78282F23
:1036800000D14561CF78482F00D10561761C082E06
:10369000E4D34460F0BD0000F0B5144C002801DA1A
:1036A000E36900E06368420D120185B2C0F301577F
:1036B0009540C0F30346032F05D0C2020AD503226A
:1036C000B240934307E023F07062636823F07063B5
:1036D000636002E0AB4343F0706201B12A4300280B
:1036E00001DAE261F0BD6260F0BD0000000001405F
:1036F0000246002092680A4200D0012070474161D2
:103700007047016170470AB10161704741617047BC
:103710004FF6FF62B0F57F4F04D0911C884203D171
:10372000002070471046704704490988814201D340
:10373000081A01E0101A084480B270478808002077
:103740000148008870470000880800200F4A104B8D
:1037500092F838105B5C834201D1012004E00D4BEC
:103760005B5C834203D1002082F83A0070470A4B29
:103770005B5C834201D18120F6E7084B595C8142B2
:1037800001D18020F0E70320EEE70000380100209F
:10379000A0B80008B2B80008A6B80008B8B8000879
:1037A0000A4810B501784FF000024C0708494FF065
:1037B000FF0389684FEA017105D5002901DA827299
:1037C00010BD837210BD0029FBDBF8E73801002033
:1037D000A4020020F0B5194E194C0022E31CA6F1FA
:1037E000060CB75CA518ED78FF5C0D430F43BD4296
:1037F0001FD01CF80270FF5C0F43BD4219D0154664
:103800000023A618F6780E43C6545B1C1CF8022051
:10381000DBB2062BF5D3C17881700179C17000212C
:103820004218491C15711CF80550C9B20629F7D376
:10383000F0BD521CD2B2032AD3D3F0BD7AAF000838
:103840005804002010B502460021064B06205C18E3
:103850006478944200D10846491CC9B20629F6D3BF
:1038600010BD0000380100200548D0E900218A423F
:1038700002D14FF0FF30704700EB011080687047B5
:10388000A010002070B5164C05464FF0FF36D4E965
:103890000010814221D004EB0010806868606068ED
:1038A00004EB0010007B00F00F02AA7204202872C3
:1038B000606804EB001105F10B000E31FCF763FCAE
:1038C00072B66068401C6060402801D300206060D0
:1038D00062B6A87A08B1002070BD304670BD000005
:1038E000A0100020284810B580784FF00002C107D2
:1038F000264843D026498988F1BB2649254B40F606
:10390000B834496CB3F87630A14232DD22490978E7
:1039100079BB90F84A1061B32049C9790C0628D5C3
:1039200001F07F015A2924D290F82B11491CC9B209
:1039300080F82B11C8291CD380F82B210146D0F820
:10394000304191F82C11A34203DD052908D2491C0E
:1039500001E041B1491E80F82C11C9B2052902D3FA
:10396000012180F82A11191B084C343CE162C0F88F
:103970003031B3F5FA6F00E000E003D280F82A217D
:1039800080F82C2110BD00008F070020A402002029
:10399000E2050020380100203F070020AF0700208B
:1039A0004FF4C042C260002181620E22028241F2C5
:1039B00062024261082202834FF4604242838183A3
:1039C0004FF07842C0E9082140F6C41101807047E9
:1039D000B0F90010B0F90220891A41604269037EF3
:1039E0004A431A41836A13448362426A934200DD68
:1039F0008262836A026A934200DA8262C268836AE0
:103A00004A43017C0A410B41D118B0F91C208A427B
:103A100001DA10467047B0F91A008842FADC08B2A1
:103A20007047000010B514481449B0F894200B8872
:103A30009A1A92B2B2F5437F1DD90988A0F8941062
:103A4000B0F8921020F8601F002242860C480D4CFE
:103A5000C2888280C180C38983812489891AA4B2E3
:103A6000C4818160E11A0161074A818AC182928A18
:103A70008282511A816110BD380100204807002060
:103A8000200E0020380500204C00002009480A497B
:103A9000B0F8B2200B889A1A92B241F684639A4227
:103AA00006D3098820F8B21F418881800021418017
:103AB0007047000038010020480700200D480178B9
:103AC000C90702D00C49098801E04FF6FA71416636
:103AD000094901201039088007482438018841F03D
:103AE0000101018004481838018821F01801018083
:103AF0007047000038010020240400400A49D1F832
:103B0000982012B1521EC1F8982031F8922F521C01
:103B100021F81A294A6A521C4A628A8F521C8A87E3
:103B200001F8400C70470000380100201CB52D48FA
:103B300090F83B3090F83C20934252D000248DF80E
:103B4000044053408DF800309DF800300122012BD5
:103B500008D09DF80030022B09D09DF80030042BCE
:103B60000AD00DE01F498DF80420443108E01D49BA
:103B70008DF80420463103E01A498DF804204831BD
:103B80009DF80420012A2CD190F83D309DF800408A
:103B9000154AA34217D090F83E309DF800402342CA
:103BA00008D0B0F84C30A0F84A300B881488E31ADB
:103BB000A0F84C3090F838302BB1B0F84030148871
:103BC000E31AA0F8423012880A80A0F8402010F8CA
:103BD0003E1F9DF80020114300F801199DF80010C8
:103BE00001701CBD580400204807002070B5344DFA
:103BF00040212846FFF77CFD840080212846FFF7FE
:103C000077FD44EA4004A9152846FFF771FD0443F7
:103C1000E1B22C4C94F878508D4250D04D4084F84D
:103C20007810012D03D0022D01D0042D47D194F836
:103C30007C00A84384F87C0094F87B20AA420FD033
:103C400084F87B5094F87A2001238B401A4207D1E4
:103C50001A4384F87A2094F87910491C84F8791072
:103C600094F87910042928D330B1012811D0022802
:103C70000FD004280DD012E01348C18821F0400174
:103C8000C1802078002184F83B1020F06000207073
:103C900005E0217841F02001217084F83B000B49B8
:103CA00094F83B0091F82720904204D081F8270037
:103CB00007492020087000F00DF884F8545070BDBA
:103CC0000010014038010020000C0020580E002098
:103CD0003C07002070B50D4D40212846FFF708FD38
:103CE000840080212846FFF703FD44EA4004A9151B
:103CF0002846FFF7FDFC04430548072100F8784FEC
:103D00000171002141708170C17070BD00100140CF
:103D10003801002070B5344890F83A10CA43920731
:103D200061D001F0030280F8392090F83D305B0645
:103D30001B0E80F83D30012A01D0812A02D15B1C84
:103D400080F83D300278D2074DD0DBB203F001029B
:103D5000C3F34004A24246D1B0F856400025641C8B
:103D6000A0F85640204CA0F8585090F83E60A47A35
:103D7000B24202D080F83E200DE0A607B6EB837F6A
:103D800002D080F83F5006E090F83F30642B02D21A
:103D90005B1C80F83F3090F84030642B0CD25B1CE9
:103DA000DBB280F84030022B06D204F001039342CC
:103DB00002D1022280F84020012901D0002912D12D
:103DC00090F83820416E00EB820291610163D0E9E6
:103DD00006121144D0E908231A441144826A11449E
:103DE000C26A1144416370BD38010020FEE7000043
:103DF0002DE9F04F00BF00209E4E9F4AA6F512719C
:103E0000A6F5BE79A6F1440B06F1440E804601F5F5
:103E1000E074A1F1780301F5457A1D5C15F0C00747
:103E200006D0402F51D0C02F77D0802F76D004E11C
:103E300015F01F0504D0154440F080072F7201E0F3
:103E400082F80880012826D0022824D0032822D016
:103E5000042820D008281ED010281CD0874D55F8E3
:103E600020C0DCF8005054F820703D40CCF80050E1
:103E7000824D55F820C0DCF8005056F820703D43C4
:103E8000CCF800501D5CAD0659F820502F6813D5B2
:103E90003AF810C03EE051F820502F6854F820C086
:103EA00007EA0C072F6051F820502F6856F820C001
:103EB00047EA0C072F60E5E7DFF8B8C10CF1F00C1A
:103EC0005CF820C007EA0C077EE015F01F0504D05F
:103ED000154440F080072F7201E082F80880012825
:103EE0001DD002281BD0032819D0042817D0082879
:103EF00015D0102813D0614D55F820502F6854F874
:103F000020C007EA0C072F605C4D55F820502F6841
:103F10005BF820C047EA0C0756E00BE056E051F88A
:103F200020502F6854F820C007EA0C072F6051F882
:103F30002050ECE715F01F0505D0154440F0800730
:103F400085F8217001E082F82180012825D002281F
:103F500023D0032821D004281FD008281DD01028E2
:103F60001BD0464D55F820C0DCF8005054F82070A6
:103F70003D40CCF80050414D55F820C0DCF80050D1
:103F80005EF820703D43CCF800501D5CAD0615D5A1
:103F90003A4D3AF81070CC3514E051F820502F68A3
:103FA00054F820C007EA0C072F6051F820502F6802
:103FB0005EF820C047EA0C072F60E6E72D4D3AF87F
:103FC0001070E03D55F820502F6036E015F01F05C9
:103FD00005D0154440F0800785F8217001E082F893
:103FE0002180012830D002282ED003282CD004288C
:103FF0002AD0082828D0102826D0204D55F820C0D7
:10400000DCF8005054F820703D40CCF800501B4DB7
:1040100055F820C0DCF80050164F883757F820704C
:104020003D43CCF800501D5CAD06B1D4114F3AF8B9
:104030001050E03F57F820703D60401CC0B211287E
:10404000FFF4EBAEBDE8F08F51F820502F6854F824
:1040500020C007EA0C072F6051F820502F68DFF8C6
:1040600014C00CF1880C5CF820C047EA0C072F60E4
:10407000D9E7000074B60008E805002070B4000815
:104080004FF40771C1824FF45861018340F6145117
:1040900081837047F0B5C48AB0F900608681B0F9B9
:1040A0000250C581B0F904300227002101220382A9
:1040B000AB4204DBB54202DDC78042810CE0B34273
:1040C00004DBAE4202DDC78041811CE09D4205DB7E
:1040D000B34203DDC2804781018115E0B54204DBB4
:1040E0009E4202DDC280418105E0AE4205DB9D4279
:1040F00003DDC1804281078106E09E4204DBAB42C2
:1041000002DDC18047810281C388458900EB4307F6
:1041100000EB4505BB89AE899B1B0FFA83FEA0F817
:1041200012E00689AB8900EB460CBCF80CC0A3EB8F
:104130000C038382B0F91830B7F90CC0A3EB0C0C58
:10414000B4EB4C0F04DA80F82010A3F1A10113E0C6
:10415000A64503DD80F82010B9890BE026B1012EB9
:1041600004D0022E10D004E0062100E0052180F8E2
:104170002010A989091B6D31418309B2B1F5586F2F
:1041800004DB5B1E438304E00421F0E7002900DC2C
:104190004283418B8183F0BD0B49002288760A62FD
:1041A000CA614A62094A32F9103002EB40028B625E
:1041B000B2F90220CA62064A32F810000882A1F859
:1041C0006000A1F862007047F0010020CAB8000842
:1041D000BEB800082DE9F05FFA48FB4982880B88D9
:1041E0009A1A92B20F2A45D309888180F7498246EC
:1041F000F74D0888F74F4FF00108002678B3401EAE
:104200000880EE73F449EE622868B1F902104307A2
:1042100042F6AA2218D4FB8843F40053FB80EE4BED
:104220001B789B0709D5AB6823F08003AB60A5F82A
:10423000806085F8826085F88360C30404D485F8C3
:10424000F480C5F8F06003E085F8F460430707D414
:10425000914205DB85F8F880A5F8F66004E010E0EF
:1042600085F8F860430703D4914201DBC00703D00F
:1042700085F81561BDE8F09F85F81581A5F81661F0
:10428000F8E7B5F81C0143F69821884202D2401C99
:10429000A5F81C0102F03CFADFF84093DFF824B3E4
:1042A00099F85000ABF1180B10B1FEF705F905E0D5
:1042B0009BF8001021F001018BF80010FFF712FBB2
:1042C00000F016FAC64841F26802416C4FF40060F3
:1042D000914201DBC34A04E0B1F57A6F02DAC14AC8
:1042E000121D1060BD48DFF8E8920A2490F85100D2
:1042F000DFF8F4C2C007A9F1340938D09CF80E00E9
:10430000802802D32878800705D5B8480078C206EF
:1043100001D4800627D5EA7B89F80720AE4A4846B3
:10432000137823F002031370ABF802609BF800309F
:1043300023F001038BF80030BA7952060FD482893A
:10434000B2F5FA7F03D2521CA9F80C200FE040F618
:104350003C70814201DD002467E0042465E0002414
:10436000A9F80C6061E089F80360A9F80C60A868FE
:10437000020501D5082458E0984A92F83FE05FEA28
:10438000CE7247D0EA7B89F807209CF80930802B51
:1043900045D3974B9B781B0641D52B785B0732D4CE
:1043A000FB889B0404D500BF20F02000A86031E00A
:1043B000ABF802609BF8004040F0200024F00104BC
:1043C0008BF80040A8609CF8170080280BD300F001
:1043D0007F044FF00040DCF80030E040034202D19F
:1043E00085F8048000E02E712879C00702D15FEAC9
:1043F0008E7005D50324032A17D089F80A8014E0AB
:104400000024EE6211E020F02000A860F88820F47B
:104410000050F88095F82A01012805D005E02A68A7
:1044200042F004022A60BFE7092408B2714903F090
:1044300027FB6749704DCA6A50438013A1F8E80012
:104440000A2C6ED16A488078800602D5FCF710FDF0
:1044500009E05F488168CA0502D521F0080101E042
:1044600041F0080181605A484FF4005E41F6E123B3
:1044700090F84AC042F266614FF48042BCF1010FED
:1044800020D0BCF1020F30D0BCF1030F95F800C072
:104490005A4CCCF3810C3DD043F6FE78BCF1010FB1
:1044A00040D0BCF1020F3DD0A0F81821A0F8482060
:1044B00047F23C3CA4F800C0484C94F87040012CF2
:1044C00033D03DE02C78C4F38104012C07D0022CBA
:1044D00008D0A0F8183100BFA0F84810ECE7A0F809
:1044E0001811F9E7A0F818E1F6E72C7842F6CC4C61
:1044F000C4F38104012C0AD0022C08D043F2EB143F
:10450000A0F8184143F69914A0F84840D4E7A0F861
:1045100018C1F7E7A0F81821A0F8482046F6547C07
:10452000C8E774E0A0F81881C0E72C78C4F38104D0
:10453000012C0CD0022C0DD0A0F81831A0F8481096
:104540009BF80030DB0708D0BBF8103007E0A0F87C
:104550001811F3E7A0F818E1F0E71F498B88AAF8D3
:10456000123019B2B0F948305943C1F38F3349467C
:10457000A9F81830934200D90A83214A1278D2064A
:1045800005D50B8B41F23332934200D20A83028964
:10459000C2F3C003C2F30022934205D10B8B41F654
:1045A0009912934200D90A83164A9278D20700D111
:1045B0000E83B9F81810C162002927DD12480224C1
:1045C000067024E0C80A0020480700204A0700209F
:1045D000A4020020000C0020E2050020580E00205C
:1045E00038010020100C0140E8050020AF07002032
:1045F0008F070020C4AE0008D00400203001002046
:10460000100700207F0700205C07002000249AF894
:104610001A0098B9022C30D084B11B4801788B065F
:1046200008D5BB795B0605D5184B1B78DB0963F30E
:1046300086110170F88820F40260F8801248406CFE
:104640004E2815DBFB88180612D5B9F81610491C40
:1046500089B2A9F81610B1F5FA6F04D3A9F816605B
:1046600023F08000F8800A48017821F002010170EF
:1046700008488AF81A40C473FCE5288F0028CCD17A
:1046800043F698202887C8E738010020100700204B
:10469000E2050020A402002070B500230C8863F31B
:1046A0000F02012505FA03F6344206D0C3F10F06C6
:1046B00005FA06F1114361F30F025B1C102BF1DBCD
:1046C000028070BD70B500230C7863F307020125EA
:1046D00005FA03F6344206D0C3F1070605FA06F1DF
:1046E000114361F307025B1C082BF1DB027070BD04
:1046F000F0B5204890F866101F480129836823F41C
:10470000006234D11D49CE88740630D41C4D1F057B
:104710004FF00004B5F9025020D41A4A526C642AB2
:1047200011DC40F6386295420DDAB2040BD40278FF
:10473000520710D4B0F8D82040F6B835AA4203D2B8
:10474000521CA0F8D820F0BD43F400628260D00172
:10475000F9D44C81F0BDA0F8D840F0BD41F2CD03B2
:104760009D42FADD897AC907F7D18260F3E782605A
:10477000F0BD0000580E0020A4020020000C002014
:10478000E205002038010020F0B5364D364F0446D2
:1047900095F83B0097F83B1023780843EE1C6278AD
:1047A000834205D1E0781146FEF7E6FE207908E065
:1047B00094F802C084450CD1E1781046FEF7DCFE87
:1047C000E07905F82F0F2878805D6870287BE877FE
:1047D000F0BD82421DD161461846FEF7CDFE95F828
:1047E0004E1095F83B00814207D1B97A09B1A17901
:1047F00000E0617985F82F101EE06978012901D069
:10480000A17922E0617927E0297841F0040129703B
:1048100012E0E1788142DBD119466046FEF7ACFE3A
:1048200095F84E1095F83B0081420AD1B97A09B14A
:10483000617ADFE7217ADDE715F82F1F895D69705E
:10484000C5E76978012906D0617A85F82F10B97A11
:104850000029F1D1D8E7217A85F82F10B97A0029FB
:10486000EAD0D1E758040020380100200B48017835
:1048700021F0020100F8381B002100F818194177D7
:10488000817733218185418508214184012100F808
:104890001F1C034880F8391070470000580400209E
:1048A000380100200D4900B50B4851F8012F40F8A0
:1048B000032F89888180084801210930FEF78AFF8B
:1048C000054802211330FEF785FF034804211D30FF
:1048D0005DF804EBFEF77EBF58040020380100208D
:1048E000094944F648000880091D46F6480008803A
:1048F000091D41F2111008800348001F018841F092
:104900002001018070470000182C01402DE9F0477C
:10491000664C674B0025A0780126654A10330528B0
:104920007ED2DFE800F00313113E1100108820F062
:10493000010010801D805F480580001F0580001F5A
:104940000580FFF7CDFFA670BDE8F087594941F615
:10495000CC401C390880574945F658002439088056
:10496000091D46F658000880524920202839088041
:104970000020401CC0B27328FBD3FFF7B1FF4C49A5
:1049800084F85C502C3147F6906008804848143019
:1049900006801D80108840F0010010800220A07069
:1049A000D2E700215FF0010004EB410204EB400379
:1049B000B2F85020B3F850309A4200D20146401C61
:1049C000C0B20628F0D33C48405C84F83900FFF7B9
:1049D0004DFF1D2000F0B0FD00F076F8374E38484E
:1049E0004FF4807996F83B10012904D002291BD09E
:1049F000042930D047E040218046FEF779FE870049
:104A000080214046FEF774FE47EA4007494640468B
:104A1000FEF76EFE074347F0010084F83B0000E01C
:104A20003DE0224809302CE040218046FEF760FE40
:104A3000870080214046FEF75BFE47EA4007494673
:104A40004046FEF755FE074347F0020084F83B005E
:104A50001648133015E040218046FEF749FE8700D6
:104A600080214046FEF744FE47EA4007494640465B
:104A7000FEF73EFE074347F0040084F83B000B4876
:104A80001D3003F0FDFA94F82F0086F838001D2041
:104A900000F068FD0420A0700A48057054E71088F3
:104AA00020F0010010801D80A5704DE75804002003
:104AB000000800403C2C014080AF00083801002075
:104AC000001001403F0700202DE9F041344C14F85C
:104AD0002F0F344DE07240212846FEF709FE860074
:104AE00080212846FEF704FE46EA4006AF15394607
:104AF0002846FEF7FDFD0643207BF1B22F3C8142A4
:104B000015D084F83C0040212846FEF7F1FD8600D0
:104B100080212846FEF7ECFD46EA40063946284645
:104B2000FEF7E6FD064384F83B60FEF7FFFF1E4DEF
:104B300095F83B00012827D0022828D0042829D046
:104B4000174894F83B102730085C04F8300F14F82D
:104B50000109FEF777FE04F82F09A87A00B10120B9
:104B6000607001F07DFE94F84E0094F83B1088428E
:104B700006D094F83800062802D2401C84F8380089
:104B800084F84E10BDE8F0810548093004E004487F
:104B9000133001E002481D30BDE8F041FFF7F4BDDD
:104BA000580400200010014038010020FF2801D9DE
:104BB000FF207047C0B270472DE9F0414A4991F893
:104BC0007200AA2874D191F87300552870D1474C0F
:104BD00000200A5C2254401CC0B27428F9D3444E11
:104BE0002069C6F80100A08AA6F80500D4F81600CE
:104BF000F060D4F81A003061D4F81E0012347061ED
:104C000003F0E4F93B49608A888103F0F9F9207DDB
:104C1000123CC007307802D040F0040001E020F0E0
:104C20000400354930704FF480400861334D14F86A
:104C3000280F334985F82000608B6880A08BA880FE
:104C4000E08BE880208C2881608C688194F82400B7
:104C500081F8D60014F8010C86F83B000027C6F84E
:104C60009C70FFF71FFE2748A18E0183E18E4183D0
:104C7000218F818394F84210283C012908D0022911
:104C800001D0032909D0297821F00C01083107E06F
:104C9000297821F00C01091D02E0297841F00C016E
:104CA000297094F8642018491AB101224A8101E060
:104CB0000EE04F8194F8701001290BD094F86D101C
:104CC00059B101290CD04FF4805100BFA0F87610E3
:104CD000BDE8F08144F21C71F8E74FF40051F5E7AC
:104CE00041F25551F2E7000000FC0008580E002088
:104CF000380100204C000020F80D0020D0040020D6
:104D0000A402002038050020000C002010B5FCF79C
:104D1000FFFCFE48FE4AFF49807AC00703D088782E
:104D200020F0010005E09078800703D0887840F0FB
:104D300001008870F8480B7803704B7843708B78CB
:104D40008370CB78C3700B7903714B7943718B7986
:104D50008371C979C171EF49083109780172ED4950
:104D6000083149784172EB49083189788172E94903
:104D70000831C978C172E749083109790173E549F9
:104D8000083149794173E349083189798173E149EF
:104D90000831C979C173DF49103109780174DD49DF
:104DA000103149784174DB49103189788174D949CF
:104DB0001031C978C174D749103109790175D549C5
:104DC000103149794175D349103189798175D149BB
:104DD0001031C979C175CF4918310B7803764B78FA
:104DE00043768B788376CB78C3760B7903774B79D0
:104DF00043778B798377C979C177C6490F390978A9
:104E000080F82010C3490F39497880F82110C14932
:104E10000F39897880F82210BE490F39C97880F897
:104E20002310BC490F39097980F82410B9490F398A
:104E3000497980F82510B7490F39897980F826100B
:104E4000B44920310B7880F828304B7880F829302D
:104E50008B7880F82A30CB7880F82B300B7980F86B
:104E60002C304B7980F82D308B7980F82E30C97931
:104E700080F82F1000F1D001097880F8301000F18F
:104E8000D001497880F8311000F1D001897880F89C
:104E9000321000F1D001C97880F8331000F1D00150
:104EA000097980F8341000F1D001497980F8351083
:104EB00000F1D001897980F8361000F1D001C9796C
:104EC00080F8371000F1D001097A80F8381000F12D
:104ED000D001497A80F8391000F1D001897A80F840
:104EE0003A1000F1D001C97A80F83B1000F1D001EE
:104EF000097B80F83C1000F1D001497B80F83D101F
:104F000000F1D001897B80F83E1000F1D001C97B0F
:104F100080F83F1000F1D001097C80F8401000F1CA
:104F2000D001497C80F8411000F1D001897C80F8E3
:104F3000421000F1D001C97C80F8431000F1D0018B
:104F4000097D80F8441000F1D001497D80F84510BA
:104F500000F1D001897D80F8461000F1D001C97DB3
:104F600080F8471000F1D001097E80F8481000F168
:104F7000D001497E80F8491000F1D001897E80F887
:104F80004A1000F1D001C97E80F84B1000F1D00129
:104F9000097F80F84C1000F1D001497F80F84D1056
:104FA00000F1D001897F80F84E1000F1D001C97F57
:104FB00080F84F1000F1F0010B7880F850304B78FA
:104FC00080F851308B7880F85230CB7880F85330AD
:104FD0000B7980F854304B7980F855308B7980F814
:104FE0005630CB7980F857300B7A80F858304B7AAE
:104FF00080F859308B7A80F85A30CB7A80F85B3061
:105000000B7B80F85C304B7B80F85D308B7B80F8CD
:105010005E30CB7B80F85F300B7C80F860304B7C5F
:1050200080F861308B7C80F86230CB7C80F8633014
:105030000B7D80F864304B7D80F865308B7D80F887
:105040006630CB7D80F867300B7E80F868304B7E11
:1050500080F869308B7E80F86A30CB7E80F86B30C8
:105060000B7F80F86C304B7F80F86D308B7F80F841
:105070006E30C97F80F86F10264950310B7880F868
:1050800070304B7880F871308B7880F87230CB7844
:1050900080F873300B7980F874304B7980F8753074
:1050A0008B7980F87630C97980F87710117880F89C
:1050B0008010517880F88110917801F0030180F818
:1050C0008210117980F88310517980F884109179D9
:1050D00080F88510D17980F88610117A80F88710D1
:1050E0000C4938310A7802F0030280F888204A78A7
:1050F00080F889208A7880F88A20CA7880F88B2006
:105100000A7980F88C204A7908E00000000C002021
:10511000101000207F070020000F002080F88D2055
:105120008A7980F88E20C97980F88F106B490A78C7
:1051300080F890204A7880F891208A7880F8922030
:10514000CA7880F893200A7980F894204A7980F808
:1051500095208A7980F89620C97980F897105F4960
:1051600008310A7880F898204A7880F899208A785F
:1051700080F89A20CA7880F89B200A7980F89C20D1
:105180004A7980F89D208A7980F89E20C97980F834
:105190009F10524918310A7880F8A0204A7880F888
:1051A000A1208A7880F8A220CA7880F8A3200A7902
:1051B00080F8A4204A79C2F3400363F35F0280F8C9
:1051C000A5208A7980F8A620C97980F8A7104349DC
:1051D00020310A7802F0010280F8A8204A7880F88D
:1051E000A9208A7880F8AA20CA7880F8AB200A79AA
:1051F00080F8AC204A7980F8AD208A7980F8AE201A
:10520000C97980F8AF10354928310A7880F8B02084
:105210004A7880F8B1208A7802F0030280F8B22040
:10522000CA7880F8B3200A7980F8B4204A7980F8E7
:10523000B5208A7980F8B620C97980F8B710274957
:1052400030310A7880F8B8204A7880F8B9208A7816
:1052500080F8BA20CA7880F8BB200A7980F8BC2090
:105260004A7980F8BD208A7980F8BE20C97980F813
:10527000BF101A4938310A7880F8C0204A7880F87F
:10528000C1208A7880F8C220CA7880F8C3200A79C1
:1052900080F8C4204A7980F8C5208A7980F8C62031
:1052A000C97980F8C7100D4940310A7880F8C820C4
:1052B0004A7880F8C9208A7880F8CA20CA7880F8AD
:1052C000CB200A7980F8CC204A7980F8CD208A79E1
:1052D00080F8CE20C97980F8CF1010BDBF0700201C
:1052E0007CB50121082000F083FC4FF40050ADF89C
:1052F000040010248DF8074001208DF8060001A954
:105300001548FEF777F90121092000F071FC012111
:105310001248FEF7C1F90820ADF8000004208DF80E
:1053200003000F4E03258DF8025069463046FEF704
:1053300061F908213046FEF7E2F9ADF800408DF83A
:1053400003408DF8025069463046FEF753F91021AC
:105350003046FEF7D4F97CBD001401400002300055
:10536000000C0140FEE7000038B50121082000F0E4
:105370003FFC4FF44060ADF8000048208DF803007A
:1053800003201B4D8DF8020069462846FEF732F9CE
:1053900029152846FEF7ACF9164CE9146070207008
:1053A0002846FEF7A5F9E070A070FEF7C9F9A080C5
:1053B000E080114890F84A10104849B101290BD0FB
:1053C00002290FD003290CD1C17841F0030107E075
:1053D000C17821F0030103E0C17821F00301491CE9
:1053E000C17038BDC17821F00301891CF8E70000C5
:1053F000000C014080080020A40200207F0700204C
:105400002DE9F041414D4FF480612846FEF770F9D7
:105410000446E9142846FEF76BF9DFF8F4800746E6
:10542000002598F800002E46844205D088F80040F8
:10543000FEF786F9A8F8040098F80100844209D024
:10544000B8F80400FEF764F91E2803D388F8014079
:10545000A4B3002598F802004446874203D0A77001
:10546000FEF76EF9E080E078874207D0E088FEF72B
:105470004FF91E2802D3E7701FB300266078254934
:10548000002808791FD020F002000871E278EAB104
:1054900020F0010008710DB1002E2DD155EA060053
:1054A0002AD01D4BDA7802F00300032800D903202C
:1054B000002475B103280CD2401C10E0FFE7012541
:1054C000C8E70126DAE740F00200DEE740F001001D
:1054D000E0E726B118B1012810D0401EC0B260F339
:1054E00001020E49DA7070B1012803D0022801D000
:1054F000032801D181F84A00BDE8F0818978C90606
:10550000EDD50020EBE781F84A40F5E7000C0140BB
:10551000800800208F0700207F070020A4020020C1
:10552000704700F01F02012191404009800000F106
:10553000E020C0F88011704700F01F020121914067
:105540004009800000F1E020C0F88011704700F0B1
:105550001F02012191404009800000F1E020C0F8C5
:105560000011704700F01F020121914040098000A6
:1055700000F1E020C0F800117047000070B50F2363
:10558000C47801780122F4B1144C2468457804F4FD
:10559000E064C4F5E064240AC4F10406E3408478BE
:1055A000B5401C402C4301F1E021230181F8003477
:1055B000007800F01F018A404009800000F1E020DF
:1055C000C0F8002170BD01F01F0082404809800032
:1055D00000F1E020C0F8802170BD00000CED00E07B
:1055E0000249084302490860704700000000FA05BC
:1055F0000CED00E02DE9F05F00261D20FFF791FF84
:105600006C4CDFF8B4B1A4F1B800A77E90F8381064
:10561000DFF8A8E1DFF8A8A100258F427ED0E77669
:10562000A176626A036B5A434FEA12499BF808203D
:10563000120702D51EF8012000E00A4694F812C0B5
:10564000BCF1010F09D004EB4206B6F902C0C4F860
:1056500028C0B6F90460E6620CE043F6FF7CC4E9BA
:105660000A5C90F83DC05FEACC7C01D012B102E048
:10567000052A00D1012600EB47074FF0804CBF8977
:105680003F04B7FBF3F3E361476BBCFBF7F727621B
:1056900094F813C0BCF1000F06D0BCF1010F05D087
:1056A0003B4403EBD3735B10636201E03B466762EC
:1056B000DFF810C14FF6FF7707EA8307ACF80870F0
:1056C0009AF8007090F80A8090F83DC0082F08F012
:1056D00003070CF0030C05D067450BD1B8F1000FA0
:1056E00005D008E0674505D0B8F1000F03D05B4254
:1056F000636200E06562C6B1636A002B03D006DD19
:10570000228D05E00AE0304B33F8122000E0A28D34
:10571000A4F86020227822F0200222709AF800205B
:10572000042A07D0082A05D012E0B4F8603003EB51
:105730000902EDE780F8405065629BF80800000719
:1057400001D51EF80110204830F81100A4F86000BF
:105750001E49606A09883E314843B4F8601001EB85
:10576000204006B21D20FFF7F2FE606A002807D035
:1057700021784FEA81600ADD002804DAA08D09E073
:10578000B4F8600006E0E06AB04208DB0CE00028F4
:1057900002DA208D208208E0A06AB04204DD208277
:1057A00041F02000207000E0268225756575258671
:1057B000BDE8F09FF0010020A4020020ACB8000872
:1057C0003F070020940B0020BEB8000824040040CE
:1057D00043184FF48042934210DD904202DD1046A0
:1057E00000210BE0914202DD0020114606E080031B
:1057F000B0FBF3F000B2C0F5804109B241EA0040CD
:105800007047F0B541F2F1130022C3600E248262AA
:1058100004824BF2660508264561068343F6FF774E
:105820004283878340F2492E4FEA873CC0F808E064
:10583000C0E9082CCB608A620C824D610E834A83DA
:105840008F83B4208860C1E9082CF0BD00218162FB
:105850000949C1600E210182084941610821018383
:105860004FF44041418343F6FF7181830907016290
:105870000349416270470000B6A001001C0C010002
:1058800000C0FF0F064941F68160088005480168A5
:10589000054A01F4E06111430160BFF34F8FFEE759
:1058A000442C01400CED00E00400FA05F8B501219C
:1058B0000D2000F09DF94FF4E060ADF800001824D1
:1058C0001D4E8DF8034003258DF802506946304681
:1058D000FDF790FEB1153046FDF711FF711530460A
:1058E000FDF70DFF31153046FDF709FF4FF460401D
:1058F000ADF800008DF80340104C8DF80250694659
:105900002046FDF777FE61142046FDF7FAFE4FF4BE
:1059100080412046FDF7F5FE4FF400412046FDF79B
:10592000F0FEA014ADF8000048208DF80300694691
:105930002046FDF75FFEF8BD00080140000C014065
:105940002DE9F0410121CE028CB0304600F050F933
:10595000DFF87081404601F013FC08A801F03CFE1E
:105960004FF45860ADF824000024ADF8204020200A
:10597000ADF822000125ADF826408DF8285008A981
:10598000404601F0DBFD0021404601F02EFE4FF6BF
:10599000FF71404601F033FE01220021404601F034
:1059A000BFFD0121404601F0A7FB04A801F0BFFBA9
:1059B000ADF81060A802ADF81200ADF814408120D7
:1059C000ADF816002803ADF81800ADF81A40ADF890
:1059D0001C4004A9404601F099FBADF8084008209E
:1059E000ADF80A006027ADF80C408001ADF80070FA
:1059F000ADF80440ADF80E00ADF80240ADF8064039
:105A00006946404601F07CFC6946404601F0BEFC18
:105A10006946404601F004FDADF8045040F61450CC
:105A2000ADF80070ADF80600ADF80840ADF80C40D8
:105A3000ADF80250ADF80A40ADF80E406946404658
:105A400001F032FD0121404601F07AFB0821404679
:105A500001F096FC3146404601F0D8FC0821404652
:105A600001F01CFD3146404601F050FD70214046DA
:105A700001F059FD18208DF82C008DF82D408DF87F
:105A80002E408DF82F500BA8FFF778FD0D480C30F5
:105A9000018841F0800101800A481430018841F0FA
:105AA00001010180001F04800121404601F052FBEA
:105AB0008DF828500121404601F056FB0CB0BDE89E
:105AC000F0810000002C0140704740F2134141601A
:105AD000082181608621C1604FF480410161494203
:105AE000416100210162C16270470162704700009C
:105AF00010B501884288891A09B20183B1F5005FA7
:105B000002DBA1F5804104E011F5005F02DC01F544
:105B100080410183B0F9182041685143C161836815
:105B2000846A5343C2681B12624303EB2222036A56
:105B30001A44114402628A13426241698A4203DBB9
:105B400001698A4200DC11468A1AC0E90A21028EE4
:105B50004FF40373594302EBA13202860B4A1278C9
:105B6000082A04D10A4A936F03EBA1319167B0F977
:105B70003010B1F5804F02DDA1F5804103E000292E
:105B800002DA01F58041018610BD00003F070020C8
:105B9000140C0020034A516821F440410143516034
:105BA0007047000000100240044A0029516901D0EA
:105BB000014300E081435161704700000010024042
:105BC000044A0029D16901D0014300E08143D16139
:105BD0007047000000100240044A0029116901D0FA
:105BE000014300E081431161704700000010024052
:105BF000044A0029916901D0014300E08143916189
:105C00007047000000100240044A0029D16801D00A
:105C1000014300E08143D160704700000010024062
:105C20002DE9F041274CA61540212046FDF760FDE7
:105C3000850080212046FDF75BFD45EA40053146A1
:105C40002046FDF755FD0543EDB240212046FDF706
:105C50004FFD870080212046FDF74AFD47EA4007B7
:105C600031462046FDF744FD0743F8B2A842DBD198
:105C700040212046FDF73CFD870080212046FDF7AE
:105C800037FD47EA400731462046FDF731FD07431F
:105C9000F8B2A842C8D140212046FDF729FD87006F
:105CA00080212046FDF724FD47EA40073146204683
:105CB000FDF71EFD0743F8B2A842B5D12846BDE85E
:105CC000F08100000010014010B50268416802FB3D
:105CD00002F301FB0133B3F1805F11D91B0E103BBE
:105CE0000A4C9BB212B234F8133009B25A435943EA
:105CF00042F38F3241F38F31C0E90221012102E0EA
:105D0000C0E902210021017410BD000098AE000816
:105D10002DE9F05FF848F94902880B889A1A92B287
:105D20000F2A7DD309880180F54802468189D288EF
:105D30004B0703D48B0701D4CB0702D042F4007287
:105D400001E022F40072C2808246080702D4504665
:105D5000C90604D5BAF8061041F0010102E0C18875
:105D600021F00101AAF80610E548FDF769FAE548B7
:105D7000B0F93A10B1F5804F02DA491C418703E0CF
:105D8000E0494FF480404887DFF87C9341F6CC40EF
:105D9000DE49D9F85020824203DD886820F01000E7
:105DA0008860DB48DB4E0024038823B15B1E038040
:105DB000CC73347029E0BAF8060045041DD4BAF853
:105DC0000C30DD0619D41D0717D4050615D4850639
:105DD00013D4050511D4450603D5CF4D2D782D06D6
:105DE0000BD5450709D4C50507D4050705D4850497
:105DF00003D4C00601D4D80707D0C848CC73C84B19
:105E00003470C4831C8080F828408B46B1F842105F
:105E1000DFF81083C44869B1491EABF8421000E0B6
:105E2000DEE098F8005025F0020588F800508BF865
:105E30000F400BE098F8003043F0020388F8003080
:105E40003178012903D10178062900D134703178E5
:105E5000DFF8D8E2B64D01270A2973D2DFE801F056
:105E6000F5C005C0F4F3C072F2F102F0C5F9DFF835
:105E70009CA2A548AAF1340ABAF81C10491C8AB29F
:105E8000AAF81C20416C40F62820814202DAAAF8C8
:105E90001C4013E09B4840F6CC43C06898420DDBA1
:105EA000B8F9040043F69913984207DBB2F5FA7F7C
:105EB00004D32A7812B9AAF81C402F709D4A108882
:105EC00068B19AF804305B1CDBB28AF80430022B0C
:105ED00005D399488AF8044003885B1C03809BF82B
:105EE0000F00D846092814D040F2DC5B022879D094
:105EF000A8F83441B8F84400A146C8B141F288344A
:105F00004846AAF81C90A14221DA297801291AD022
:105F10001DE079484430FDF743FDFDF707FA7A4864
:105F2000416CCAF8301041F27C51CAF8201069E285
:105F3000A88AA8F83400E86A6863A86A2863A8F801
:105F4000447037E0A0E17C492870088010807B49CC
:105F5000C978B7EB511F08D098F82C2102B97848BE
:105F6000C8F8DC0088F8EE7005E0C8F8DC0088F8B6
:105F7000EE00CAF82800B7EB511FB8F9341040F60C
:105F80003A2001F21D520AD08242B8F8DC0000B279
:105F900002D810231A4609E02023022206E082429A
:105FA00001D8102300E020231022002000F0A6FBDF
:105FB000A8F83400614863494FF49A73C078B7EB8E
:105FC000501F51480FD0426C5A4509DAB5F90A0002
:105FD000984205DC86F8009088F8EE90A1F81A90B7
:105FE000BDE8F09F19E0406C584503DAB5F90A2086
:105FF0009A42EFDDB8F8442040F6C413521C92B226
:10600000A8F844209A42E5D23E4AD268002AE7DC4A
:1060100042F6E0629042DDDAE2E7B8F8342140F679
:10602000B830824207D2344B183B1B78DB0702D1D1
:10603000521CA8F8342193B25B4507D842F6CC40F5
:1060400008E0B6E094E0DBE0D6E0DEE0A8F834015A
:1060500043F26660E867CAF830108AF809703A4E71
:10606000A8F8444088F8EE40707F5546F0B1F07FC4
:1060700088B3B8F82C00B8F9341000B20A2305220E
:1060800000F03CFBA8F83400F4777477B8F91A01F3
:10609000B8F91811884229DA697901F1010111F082
:1060A000FF01697156D06C71401C21E04FF48040B3
:1060B000A8F8E800D8F82C10814200DA08462349F5
:1060C00000B2688391F84D100029B8F9341003D05C
:1060D0003623052203E005E040F24713362200F0A4
:1060E0000DFB00E0A320A8F83400CFE730DD801ED0
:1060F000A8F81A012EE00000C80A00204807002076
:10610000000C00203805002038010020A4020020E7
:106110004C0700203F07002010070020300A002015
:1061200006000020E2050020400700205802002061
:106130004C000020080000200A000020A7070020D3
:106140009AF9FFFF3C0B0020200E0020580E002083
:10615000A8F81A11B8F934004FF48041884202DDE2
:10616000A8F834103CE70028FCDAA8F8344037E7F8
:10617000D84ADBF8E0105846914202D2491CC0F8D8
:10618000E010C17B082903D1D0F8E01091420CD374
:1061900034708168CA0502D521F0080101E041F0A0
:1061A00008018160CBF8E0401AE7BDE8F05F02F03B
:1061B00097BF9BF80F005F46092803D0BC868BF879
:1061C0000F4061E1C44D686A401C6862022809DD25
:1061D000288E012301B2288C052200B200F08EFA2D
:1061E0006C622863BD48298E0180B9F84410418053
:1061F000FDF7EEFBB886F3E6BDE8F05F04F0ECBC1B
:106200009EF8000009287DD0EAE68BF811419BF842
:106210002C3163B142F31101CBF8DC40B04A8B035F
:10622000E962891093628A03A962AE498A62AA4927
:106230008C83D9F8442041F288318A4207DA2978E0
:10624000012904D1A8492C700C80A8490C80A84AC7
:10625000DFF8A0C21188491C8BB2A7491380C82B54
:1062600004D391F80080B8F1010F19D0B3F57A7F0B
:1062700004D391F80080B8F1020F11D0B3F5FA6F92
:1062800002D30B78032B0BD09BF80F10891E082923
:106290007ED2DFE801F010B9FBF7047D85AB9FE605
:1062A0000C701480BAF8062022F40062AAF80620C6
:1062B0008CF80070E8E7D9F84410C846822904DA5F
:1062C0000178062901D00470F5E0FDF769FA98F825
:1062D0000000400613D58948807804280FD0D8F8EC
:1062E0004410404682290ADA817A98F83D0001F08C
:1062F000030100F00300814201D001F02DFEB14600
:10630000307800E0C0E00628C9D088F83F40D8F8CF
:106310005000734940F311008203E86280108A62E2
:106320008103A8626F4846468162FCF7FFFF6A4816
:106330005D464772BBF81801ABF81A01706CABF8F8
:106340008640B0F5437F10DD4FF48040A5F884000F
:10635000A86840F48060A86096F8381005299ED19E
:1063600040F01000CBF8080016E04FF48041A5F88B
:106370008410A96821F48061A96040F28A218842D2
:1063800004DA3078400601D402F098FDA86800E0F5
:1063900098E040F01000A860022089F800001FE695
:1063A000D9F84410B1F5437F02DA017806298AD181
:1063B0005348017821F040010170FCF7B7FF43F624
:1063C000FE70ABF81A010BF1E005FDF7E9F94D4855
:1063D00010F8341F21F00101017042492C608C62D9
:1063E0003F498C62082131704464F9E53B48FDF770
:1063F000D7FAFCF79BFF3848D9F84410016341F203
:106400007C51016209203BE09AF80600C006C6D420
:10641000D9F844004D46B0F57A7F35DDFDF7C0F977
:106420002878400611D53548807804280DD0686C4E
:1064300082280ADAA87A95F83D1000F0030001F0EE
:106440000301884201D001F087FD85F83F40B5F88F
:106450005000ABF8340001B24FF480405C468142FA
:1064600000DDA086FCF762FFA06840F48060A060B9
:1064700095F83810052992D140F01000A060022054
:106480003070ADE514E001E03470A9E5D9F84410AE
:10649000B1F5437F02DA0178062988D1BAF80610EF
:1064A00021F02001AAF80610FDF77AF90420E7E7A9
:1064B0000078062801D0377092E509208EF8000098
:1064C0000520DDE70D498C70047085F85E40ABF85F
:1064D000344085E5C0D40100700200200C0B002080
:1064E000000A0020D00900200A0000200800002037
:1064F000100100200E01002012010020580400208D
:106500004E070020140C002030B585B00121042076
:10651000FFF76EFB4FF40040ADF8100048208DF8F7
:10652000130004A91848FDF765F801210846FFF794
:1065300047FB40F68C20ADF8040003240020ADF8A2
:106540000040ADF80200ADF806004FF08045694606
:10655000284600F0F3FF1C208DF80C008DF80D404C
:106560008DF80E4001208DF80F0003A8FFF706F804
:1065700001221146284600F0BBFE0121284600F00A
:10658000E9FD05B030BD0000000801407047000083
:106590002DE9F041304CE07800285AD120780028CD
:1065A00057D0401E10F0FF00207052D14FF496706B
:1065B000208272B6294F45F2AA50A7F87200002037
:1065C000FCF792FE264D13202860FCF79FFEA8BB27
:1065D0003420E86002202861224E6E61286940F074
:1065E00040002861FCF792FE40BB00211E4A08468D
:1065F0005FEA255312F800C0BCF1FF0F00D0012163
:10660000401C80B29842F5D3C1B9C4E90676392658
:106610000127A06910F8011B10F8012BA061E069A7
:1066200001EB022102886A612F6120F8021BE06100
:10663000FCF76CFE10B9761EB6B2EAD20120FCF768
:1066400053FE62B601F0DCFC0848816821F4804109
:106650008160BDE8F08100003C070020580E00205A
:106660000020024000FC000800FC0008A4020020FA
:106670001948016841F010010160016821F003012F
:106680000160016841F00201016014484168416005
:1066900041684160416841F480614160416821F492
:1066A0007C11416041680E4A11434160016841F02C
:1066B0008071016001688901FCD5416821F0030106
:1066C0004160416841F0020141604168C1F38101CC
:1066D0000229FAD170470000002002400010024059
:1066E0000000280830B5044C039D6080A180E28042
:1066F0002381658130BD0000F40B00200A448242F2
:1067000001DA10B27047C91A8142FBDD08B2704746
:106710002DE9F04F4A48DFF82CA1DFF82CB1C17FFA
:10672000477A046849480022DFF82C91466C4848B3
:106730004FF0010E802985784648836834D301F0F4
:106740001F0C5AF82C100C420146096802D041F483
:10675000805101E021F4805101605FEAC14C1ED4F8
:106760005FEA814C1BD599F80AC0C8465FEACC7C29
:106770000BD05FEAC31C12D4A8F80A209BF8008053
:1067800028F002088BF8008009E0322E07DC5FEA6F
:10679000857C04D55FEA035C01D4A8F80AE04FEADF
:1067A000113C6CF34D310160802F24D307F01F079B
:1067B0005AF827100C42016802D041F0040101E0B0
:1067C00021F0040101604C0711D44C050FD599F854
:1067D0000A70FF070BD0DF0109D4A9F80A209BF843
:1067E000007027F002078BF80070C0F89C208C081E
:1067F00064F38A21016099F80A40E40719D1174C23
:1068000094F86440012C14D1322E10DC0468660721
:106810000DD51B050BD4E30409D5AB0707D5D0F87C
:106820009C304EF66024A34205D9A9F80AE0C0F8CE
:106830009C20BDE8F08F5B1CC0F89C30F9E700009D
:10684000E8050020E8B30008E20500203801002038
:106850008F070020A4020020000C0020580E00200A
:1068600010B5FAF79BFA0F48018821F00201018068
:106870000C49183109880C4A928E1144094A343265
:10688000118008490C390A8842F001020A80011D72
:106890000A884FF6ED531A400A80018841F0120130
:1068A000018010BD0C04004058040020130A03703E
:1068B0000A70704705484FF6FF620188491C89B28B
:1068C0000180914201D30021018070478808002097
:1068D0000F4810B5016841F00101016041680D4A9F
:1068E0001140416001680C4A11400160016821F4C7
:1068F00080210160416821F4FE0141604FF41F01D5
:106900008160FFF7B5FE05494FF00060086010BDDB
:10691000001002400000FFF8FFFFF6FE08ED00E067
:106920004FF0E02005494161054AF02182F8141D2D
:10693000002181610721016170470000DFA501008E
:106940000FE000E02DE9F047DFF8D4A0BAF800002E
:106950004FF00005000635D5324C6088401C608041
:10696000FBF780FDDFF8C0C0304A31489CF800706A
:10697000677092F800800723C8262E494FF005095A
:10698000B8F1010F22D02C4FB7F806C0BCF1000FB0
:1069900038D084F80090848944F008048481C48845
:1069A00024F40064C480886820F004008860FD80BE
:1069B0001370A1F8426000204FF49661401C80B231
:1069C0008842FBD3AAF80050BDE8F08777B1012FC9
:1069D00012D0C78847F40067C780886840F0040079
:1069E0008860032020708CF80090E1E7878947F0E9
:1069F000080787810120F5E7878947F0100787811D
:106A00000220EFE7042727700C4C2570C48844F45B
:106A10000064C480886840F004008860C8E7000013
:106A2000102C01402C070020400700203F070020C9
:106A3000000C0020A4020020C80A00205D070020EE
:106A4000704700002DE9F0434FF08040018A21F0AB
:106A500001010182AA48007800287CD1A94FF87B67
:106A6000002878D1A848406C322874DCA748806898
:106A7000DFF89C924104A74DB9F804004FF00004E0
:106A800003D4401CA9F8040024E1002874D029781C
:106A9000012611B1012912D013E14946B0F5BE7F9C
:106AA000FAD92E70CC718C71EC702C72287A0A187D
:106AB000401CC0B2147228720F28F7D301E1B9F854
:106AC00002204946824201D9EE7100E0EC71904803
:106AD0008A7908300F2A15D2CB79082B0BD2C3F153
:106AE0000708EB7912F800C003FA08F36344135463
:106AF000CA79521CCA71CA79082A03D18A79521CF0
:106B00008A71CC7199F80610C8460F2973D10D21EE
:106B1000FBF740FAA881010A6970C0B2A87088F832
:106B2000064098F816208A4265D198F815108142DF
:106B300061D198F80BC07849032302227748BCF151
:106B4000000F10D0BCF1010F02D0BCF1020F14D025
:106B500080F86A2000E0C7E091F800C02CF00C0C2F
:106B60000CF1080C0FE080F86A6091F800C02CF07E
:106B70000C0C0CF1040C06E0A5E080F86A3091F8EA
:106B800000C04CF00C0C81F800C098F80C10B6EB6B
:106B9000111F04D180F86E4087F84A400EE0B2EB36
:106BA000111F04D180F86E6087F84A6006E0B3EBED
:106BB000111F03D180F86E2087F84A200B0717D0E9
:106BC00001F00F01012901D0022915D080F86C6075
:106BD0002C7198F80D102A7906FA02F30B406B71AC
:106BE000082A41D2DFE802F00B0F4016212C333A7D
:106BF00080F86C40ECE764E080F86C20E8E713B3C1
:106C000080F8704030E013B180F850602CE080F8DC
:106C1000504029E023B180F8656087F8076123E0E0
:106C200080F8654087F807411EE023B187F8F940F6
:106C300080F84D4018E087F8F96080F84D6013E067
:106C400013B180F868600FE080F868400CE013B181
:106C500080F8666008E080F8664005E013B180F8CF
:106C6000676001E080F86740521CD2B22A71082A9E
:106C7000B1D398F80E108A0704D587F8F56080F82C
:106C8000646005E0264A87F8F54080F86440548146
:106C9000C90702D080F8294001E080F8296098F8FF
:106CA000111000F86D1FC2781E48012A1ED001B3D2
:106CB000012921D04FF48051A0F876101A493C20C8
:106CC0000870A9F80240A9F80440B9F80210491C5C
:106CD000A9F80210B9F80210B1F5FA7F04D940F210
:106CE000F511A9F802102C70BDE8F08344F21C7174
:106CF000E2E74FF40051DFE741F25551DCE70000D5
:106D00003F070020A40200203801002000100140AD
:106D1000400E0020C8060020D0040020580E00209D
:106D2000000C0020380500203C0700202DE9F05F12
:106D3000FCF736FD8E4D2888A5F10406C0070AD061
:106D4000308820F008003080288820F00900288052
:106D500002F0B4F8D9E02888DFF81892DFF818823A
:106D6000864C80071AD5B9F8001041F00101A9F846
:106D70000010B8F80000804914315030088028888D
:106D80004FF6F95108402880308840F004003080E8
:106D9000FEF746FF84F83C00BDE8F09F2888784F56
:106DA0004007288871D520F004002880FEF738FFBE
:106DB00094F83C108142EFD1308820F004003080FC
:106DC000FCF714FF2078410605D594F8541094F888
:106DD0003B209142E0D03978400621F00201397021
:106DE00004D5FDF771FE97F82F7004E094F83C008D
:106DF000FCF728FD0746DFF880B140F68C2A0BF13E
:106E0000180B062F47D294F83800B8423ED03846C7
:106E1000FCF79CFC2078C00716D094F83A0094F850
:106E2000391000F00302914206D0A17A00F001006F
:106E300001F00101884215D1FCF740FEF9F7FAFF95
:106E4000FCF768FF384689E0FCF738FEF9F7F2FFF7
:106E5000FCF760FF3846FCF751FE207840F0010057
:106E6000207099E7288820F008002880206B81088E
:106E700001EBD000504515D2B8F800100844ABF82B
:106E80000000308840F0080003E00DE0308820F07A
:106E90000800308080E7B9F8001041F00101A9F83E
:106EA0000010DFE75046E7E70007288831D520F0DB
:106EB00008002880308820F008003080FEF7B0FEFF
:106EC00084F83C00FCF792FE387820F0020038701D
:106ED0002078400604D5FDF7F7FD97F82F5004E021
:106EE00094F83C00FCF7AEFC0546062D08D294F859
:106EF0003800A842B5D0FCF7E1FDF9F79BFF2AE086
:106F00002048C18841F04001C180BDE8F05FFCF736
:106F1000E1BEC006288825D520F0100028803088E2
:106F200020F01000308097F838000C2802D2401C66
:106F300087F83800387840F002003870FDF7C4FD5B
:106F400097F82F50787884F8390094F83800A842E0
:106F500087D0FCF7B3FDFCF7DDFE2846BDE8F05F07
:106F6000FCF7CCBD4EF2BE110840288014E70000AB
:106F700010040040000400402404004038010020B8
:106F800058040020000C00202DE9F04F514F85B02F
:106F9000388820F0010038804E48002610300680E6
:106FA0004D4CDFF838A14FF0010894F85C0042F630
:106FB0003029C10774D072B64948816941F4007123
:106FC0008161816941F4806181614FF40040FEF785
:106FD000E1FD444D00212846F9F778FC00212846C0
:106FE000F9F76AFCDFF800B100215846F9F764FCB4
:106FF00000213E48FBF7A4FC2846F9F789FD5846D6
:10700000F9F786FD4FF46020CDE902068DF80560A2
:1070100000968DF810808DF8048069462846F9F7AF
:1070200009FE01231A460F212846F9F754FE0121D3
:107030002846F9F741FC00204946401C80B28842AE
:10704000FBD328462E600121F9F784FE28688007CB
:10705000FCD524484C30006894F85C1021F0010104
:107060002144A1F85000F9F73BFC62B6FDF738FC6B
:1070700047F69061AAF8001094F85C00401CC0B27A
:1070800084F85C000C2822D212491431A1F8008047
:10709000388840F00100388005B0BDE8F08FFFE788
:1070A000134920F00100085A12490880114945F699
:1070B0005800083908800F4846F65801001F018023
:1070C0000C4920200C390880AAF80090D4E703204E
:1070D000A070E1E700080040580400202C080040A0
:1070E0000010024000240140002801400800024036
:1070F000A4AF0008202C01400029018802D041F0F3
:10710000800101E021F080010180704710B50A88FC
:107110004B88CC881A438B8823431A430B891A4324
:107120004B8989891A430A43A0F8442010BD0021E5
:10713000018041808180C1800181418181817047CE
:107140000029818802D041F0010101E021F0010114
:10715000818070470029018802D041F0010101E0DF
:1071600021F0010101807047002930F8441F02D04E
:1071700041F4004101E0C1F30E01018070470000BD
:107180004B4910B5884202D10121C41486E0B0F108
:10719000804F09D0474988420DD101210220FEF7D6
:1071A0001BFD0021022064E001210846FEF714FDCA
:1071B000002101205DE04049884206D101210420E0
:1071C000FEF70AFD0021042053E03C49884206D125
:1071D00001210820FEF700FD0021082049E0384980
:1071E000884206D101211020FEF7F6FC0021102074
:1071F0003FE03449884206D101212020FEF7ECFC13
:107200000021202035E03049884202D10121441478
:1072100044E02E49884202D10121CC043EE02C49B1
:10722000884202D101210C0538E02A49884202D166
:1072300001214C0532E02849884206D10121402035
:10724000FEF7CAFC0021402013E02449884206D101
:1072500001218020FEF7C0FC0021802009E02049A8
:1072600088420AD1841501212046FEF7B5FC002191
:107270002046BDE81040FEF7AFBC1A49884202D153
:1072800001210C040AE01849884202D101214C0472
:1072900004E0164988420AD101218C042046FEF7F9
:1072A000B3FC2046BDE810400021FEF7ADBC10BD88
:1072B000002C01400004004000080040000C004089
:1072C000001000400014004000340140004C014018
:1072D000005001400054014000180040001C0040D4
:1072E00000200040004001400044014000480140AF
:1072F000002A828901D00A4300E08A4382817047D4
:1073000030B5028C22F001020284028C8388048B47
:1073100022F0020224F073050C882C430D891543DA
:107320004A882A43114DA8420BD0114DA84208D0DB
:10733000104DA84205D0104DA84202D00F4DA842D2
:107340000DD122F008054A8923F440732A4322F024
:1073500004058A882A438D891D43CB892B4383806A
:107360000483C9888186028430BD0000002C01405E
:107370000034014000400140004401400048014009
:10738000028B22F008020A430283704770B5028C18
:1073900022F010020284028C8488038B0D8823F46F
:1073A000E6464FF6FF7303EA052535430E8922F0C2
:1073B000200203EA061616434A8803EA0212324301
:1073C000104EB04202D0104EB04215D122F08006CD
:1073D0004A8924F4406403EA0212324322F0400650
:1073E0008A8803EA021232438E8903EA860626431C
:1073F000CC8903EA8404344384800583C9880187E7
:10740000028470BD002C014000340140028B4FF615
:10741000FF7322F4006203EA0121114301837047E4
:1074200070B5028C22F480720284028C8488838B73
:107430000D8823F073031D4322F400730E894FF669
:10744000FF7202EA06261E434B8802EA03233343F7
:10745000104EB04202D0104EB04215D123F4006657
:107460004B8924F4405402EA0323334323F4806617
:107470008B8802EA032333438E8902EA06162643E9
:10748000CC8902EA0414344384808583C9888187C7
:10749000038470BD002C014000340140828B22F037
:1074A00008020A438283704770B5028C22F480522E
:1074B0000284048C8288838B0D8823F4E6464FF681
:1074C000FF7303EA0525354324F400560C8903EACB
:1074D000043434434E8803EA06362643094CA0425E
:1074E00002D0094CA04205D122F480448A8903EAE3
:1074F0008212224382808583C988A0F840100684C6
:1075000070BD0000002C014000340140828B4FF61A
:10751000FF7322F4006203EA012111438183704763
:10752000018582827047828822F070028280828880
:107530000A4382807047A0F84010704730B5028837
:107540001B4B1C4C98420DD0A0420BD0B0F1804F89
:1075500008D0194DA84205D0184DA84202D0184DA8
:10756000A84203D122F070054A882A43154DA8424B
:1075700006D0154DA84203D022F44075CA882A438C
:1075800002808A8882850A88028598420AD0A042B1
:1075900008D00E4A904205D00D4A904202D00D4AC2
:1075A000904201D1097A01860121818230BD00001B
:1075B000002C01400034014000040040000800405D
:1075C000000C00400010004000140040004001404A
:1075D00000440140004801404FF6FF7181800021C6
:1075E0000180C1804180017270470029018802D06A
:1075F00041F0020101E021F0020101807047002901
:10760000018802D041F0040101E021F00401018071
:10761000704780092830FF2801D9FF207047C0B289
:1076200070472DE9F041B1F9025000231E240F22CA
:10763000854203DDB1F90000BDE8F081B1F97A506F
:10764000854202DAB1F97800F6E701EB8205B5F977
:107650000250854201DA134600E01446E21852084F
:107660005D1CAA42F1D101EB8203B3F902408442CE
:1076700006DAB3F9067031F92250B3F9046005E077
:1076800033F9027C31F9225033F9046C001BC11725
:1076900089013A1B41EA9061D3178001F8F742FD56
:1076A000721BA0FB024601FB0261D31700FB031013
:1076B000810641EA9410284400B2BDE72DE9F04F5D
:1076C000DFF8B8B16A48DFF8AC91DFF8ACA190F808
:1076D0000EC0BBF91A70BBF91C60BBF91850BBF99E
:1076E0006C10BCF1070F48D2DFE80CF08D041A30A3
:1076F000485E7600D9F80020C284DAF800200285BE
:10770000C28C038DA7EB820212B2A6EB83034A431D
:107710001BB2594342F3CF2241F3CF23D11870E07B
:10772000D9F800208284DAF800200285828CA5EB4B
:10773000820213B2028D4B43A6EB820212B243F3D4
:10774000CF24514341F3CF23E11814E0D9F80020AE
:107750000285DAF800208284028D838CA6EB8202F7
:1077600012B2A5EB83031CB24A43614342F3CF2319
:1077700041F3CF24191949420AB244E0D9F8002054
:10778000C284DAF800208284C28C838CA7EB820248
:1077900012B2A5EB83034A431BB2594342F3CF22F3
:1077A00041F3CF24111914E0D9F800208284DAF8CB
:1077B0000020C284828CC38CA5EB820212B2A7EB9C
:1077C00083034A431BB242F3CF24594341F3CF22F0
:1077D000A11849420BB216E0D9F800200285DAF868
:1077E0000020C284028DC38CA6EB820212B2A7EBEA
:1077F00083031CB24A4342F3CF23614341F3CF22B8
:10780000991849420CB2BBF91E50594605F21E5652
:10781000A64201DACE8306E0A5F21E55A54201DD9F
:10782000CD8300E0CC83B1F9204004F21E5595428F
:1078300001DA0D8406E0A4F21E54944201DD0C84AA
:1078400000E00A84B1F9222002F21E549C4202DABE
:10785000ABF8224008E0A2F21E529A4202DDABF8D9
:10786000222001E0ABF82230417B8173BDE8F08F2C
:10787000A40200203C2401403C280140380500209F
:107880002DE9F04704467048714E002702786F4892
:10789000022AB0F9341004D0082A6ED0092A6DD01B
:1078A000CDE0C27B022A02D1B0F844205AB1A4F83C
:1078B000421071810423B6F908101A460020FEF721
:1078C0001DFF3081BBE06349DFF88C81496A0D14EC
:1078D000E58090F84A1099B10089DFF88091C0F3F3
:1078E000C001C0F30020814223D1D8F8440040F207
:1078F000BA41884240DD40F66A1188420ADC15E050
:10790000B4F9020040F2DA21884279DD40F26A419E
:10791000884204DD0823B4F942101A464EE0A0F272
:10792000DA20F8F788FD00224D4B56E0A0F2BA406D
:107930004FE04C480078C0060CD5D8F8440041F21E
:10794000243188425CDD41F2D4718842E2DC00F6E9
:10795000DC4020E04448DFF8149190F870100129D1
:107960000DD090F86F00012809D041480178C9076F
:1079700046D04049098889B142E05AE05DE0B4F957
:10798000020041F6DC6188423ADD42F2341188425D
:1079900010DC00F59270A0F500501AE0B0F910006C
:1079A000B4F90210A0F59672914229DD00F59672A5
:1079B00091420BDDB4F9421020231A460020FEF755
:1079C0009DFEA4F84200002817DB1BE0081A00F512
:1079D0009670F8F730FD00224B46F8F798FC0E221F
:1079E000F8F704FDF8F75EFD00B2C0F5804068438B
:1079F0008013A4F84200002D04DCA4F8427001E0DA
:107A0000A4F842501C48B0F90410D8F85000081AE5
:107A1000718B01EB600000B2F082002800DCF7827D
:107A2000B4F94200B6F91610884200DB08467081AE
:107A300004E01248B0F87C00F9E77181378184F8DE
:107A40004070BDE8F08700003F070020A40200203E
:107A50004C000020380500203801002000C0924072
:107A60000000794010070020580E002000C082401E
:107A7000B00A002008000020E2050020140C0020BD
:107A80002DE9F041B1F9025000232B241522854243
:107A900003DAB1F90000BDE8F081B1F9AE508542DA
:107AA00002DDB1F9AC00F6E701EB8205B5F9025051
:107AB000854201DD134600E01446E21852085D1CC1
:107AC000AA42F1D101EB8205B5F90230834206DA10
:107AD00035F9026C35F9044C31F9221006E01E46E6
:107AE00031F92240B5F90630B5F90410801B091BA5
:107AF000C5178911AD0345EA90458703A1FB070C23
:107B0000CA1702FB07C201FB05219A1BD317F8F71E
:107B100009FB000A40EA0160001900B2B0F5804F8D
:107B2000B9DB43F6FF70B6E770B5134C40F224455D
:107B30002946204600F02CF800281BD0204600F0F3
:107B400046F82946204600F01DF80C4C002120463E
:107B5000FAF7F6FE2046FAF771FFC0F16400084913
:107B6000C0B20428087201D900F0B2F9BDE8704033
:107B7000FAF7A2BF70BD0000003801405800024073
:107B8000740600200A0A01219140C9430180704710
:107B900030B501F01F0201240025C1F3421304FA9D
:107BA00002F2012B0FD0022B0FD0838A4FEA112152
:107BB0000088134204FA01F400EA040001D000B185
:107BC0000125284630BD8389F0E7038AEEE78088E7
:107BD000C0F308007047000070B5214C2068214DAB
:107BE000400103D520492846F9F7B2FA2068000180
:107BF00004D51D492846FF31F9F7AAFA2068C000CC
:107C000003D51A492846F9F7A3FA1948194A017801
:107C1000CB0712D192F82F30012B0ED0FAF788F94A
:107C20002068C0F382611448072916D0216811F03A
:107C3000E05F01D15521017070BD012382F82F3022
:107C400021F0010101700D4801680D4A01F4E06165
:107C500011430160BFF34F8FFEE70021EBE7000007
:107C60000864004000640040010000380000013852
:107C70003E080020CC0E0020480800200CED00E05B
:107C80000400FA052DE9F04186B0002604208DF8A5
:107C90000800864C4FF48068009601968DF80A60C3
:107CA0008DF8136041462046F9F7B2FB0125012803
:107CB0001CD17F4F07F8306FF9F784F9206840F442
:107CC0000040206079481430016821F00101016012
:107CD000784E306800F0F2FD002177A001F04CFEF4
:107CE000306041462046F9F74BFA3D7002212046AC
:107CF000F9F78EFB01287DD16A4600212046F9F76D
:107D00005DFC01986F4920F0604088609DF80A2072
:107D1000082A1CD16C4A10440C2818D2DFE800F065
:107D2000060BBFBFBFBFBF1854737EA565489DF843
:107D30000B106F309DE0634B00206A461733161816
:107D4000F67A1E54401CC0B20828F8D30D70A6E085
:107D50005C499DF80B004F3103090A7860F3030278
:107D600063F30412430963F34512800960F3871239
:107D70000A709DF80C0048709DF80D0088709DF801
:107D80000E00C8709DF80F20087962F300005208B9
:107D900062F3470008719DF8100048719DF81120AA
:107DA0008879930862F3010063F38300120962F398
:107DB000071088719DF81200CA7960F30602C009A5
:107DC00060F3C712CA716AE040489DF80B10017059
:107DD0009DF80C1041709DF80D1001F003028270A7
:107DE000C1709DF80E1001719DF80F1041719DF842
:107DF000101000E057E081719DF81110C1719DF8DD
:107E0000121001724BE02F489DF80B20573001787B
:107E100062F30101920862F387012AE029499DF883
:107E20000B205F31087862F30300120962F3071038
:107E300008709DF80C0048709DF80D20887862F35A
:107E40000600D20962F3C71088709DF80E00C87052
:107E50009DF80F0008719DF8100048719DF8110001
:107E600088719DF81200C87119E016489DF80B1032
:107E7000673001709DF80C1041709DF80D108170F5
:107E80009DF80E10C1709DF80F1001719DF8101033
:107E900041719DF8111081719DF81210C17102217C
:107EA0002046F9F76DF906B0BDE8F08100640040A6
:107EB000CC0E00204C0800206465765F63616E3153
:107EC0000000000060070020FFFE00E71010002007
:107ED00070B51D4D00242878432834D16878462891
:107EE00031D1A878502807D0512805D0812803D057
:107EF000892801D0212826D1144E7071E978717239
:107F0000A81C891CFAF77EF8B072717A29440979A5
:107F10003182884217D106F10E00017841F002014A
:107F200001700B48016841F020010160317A094875
:107F3000002204E02B5D03552A55641CE4B28C42F8
:107F4000F8D38078707170BDF008002074060020AE
:107F50000C0C0140920D002070B51D20FDF7ECFACD
:107F6000FCF7B2FD1D20FDF7FDFA154890F82F1023
:107F7000144D0623144C85F8381090F83B1095F8F2
:107F80003B201143012A04D0022A07D0042A0AD038
:107F900010E0827A8A420DD0007B09E0027D8A429D
:107FA00008D0807D04E0827F8A4203D090F82000D0
:107FB000884200D12370002085F8400070BD000089
:107FC00058040020380100203F0700200B48002102
:107FD0004180A0F1B8018A898280CB891A44C2808D
:107FE0000B8A1A4402814B8A1A444281898A1144BD
:107FF000818143F6FF71C18170470000F0010020CC
:10800000084940F61C72B1F90C00904202DA00F502
:108010009F7005E041F2E302904201DDA0F59F7000
:10802000C88170474C00002038B51348C16941F041
:108030000401C1611E208DF8000002208DF80100AE
:108040008DF8020001248DF803406846FDF796FA8A
:108050000A4984200880094947F690602C3108803D
:108060000020091F0880054914310C80091F088071
:10807000081F048038BD00000010024000080040C6
:1080800030B420491E4A45788B7A114692F83B401D
:1080900091F83910AC4218D14BB10379994202D012
:1080A0004379994201D140791AE0807909E08379D6
:1080B000994202D0C479A14202D182F82F3011E056
:1080C000407982F82F0030BC7047C578AC42FAD1B5
:1080D0006BB1C379994202D0037A994205D1007AF3
:1080E00082F82F0030BCFEF7BBBB407AE9E7437A49
:1080F0009942E2D00479A142DFD0007AE1E70000A2
:108100005804002038010020FEE700002DE9F04768
:108110000446007F012868D13548E1880288511A59
:1081200089B2072916D30088E080B4F9000044F230
:10813000DD414843401346F6D96148438013A060AF
:10814000401000B2A0814FF08051B1FBF0F0F8F781
:108150006DF92061B4F90C6096B1B4F902104DF6D6
:10816000B05048430014A082B4F904704DF6B052E8
:1081700007FB02F24FEA2245E58204D4024603E0FF
:108180000020E08330E0424212B22283002D01DB66
:108190002B4600E06B421BB2DFF858906383984691
:1081A0004FF4804AB24208DAF8F737F92169F8F754
:1081B0000AF8F8F75EF9801304E0002901DA48466E
:1081C00000E05046E083B04509DA2846F8F725F983
:1081D0002169F7F7F8FFF8F74CF9801304E0002F56
:1081E00001DA484600E050462084BDE8F0870000F0
:1081F0004807002000C0FFFF2DE9F0414C484D4EDC
:1082000000250078A6F15004022806D14A4FF87BD9
:10821000022802D1B7F8440030B1A5862564B562C2
:1082200084F83850BDE8F08144488168C06849430B
:1082300000FB0010FBF78CF940F233314843810B0F
:10824000B4F8440043F6CC42504301EB903080B286
:1082500043F69911A4F84400884209D338481146DE
:10826000B0F90400884203DB97F84A00032813D0D2
:108270000123B4F934101A460020FEF73FFAA08615
:10828000B4F84000012301B21A460020FEF736FA86
:1082900020648003B06226E0B4F8460041F69A13E9
:1082A000A0F51852663A9A4209D2B4F94400214A1C
:1082B000FAF7EEFF2064012084F8380022E044F24F
:1082C0004711884212D994F83800D8B11D48017876
:1082D000491CC9B20170022914D30570206C10B179
:1082E000401E206408E084F838500BE0A0F5804080
:1082F000B0F5A47F03D2206C8003B06202E084F862
:108300003850B562B4F840000A4980B208393234B6
:1083100001F000FDB4F90000B4F9181041438913CD
:108320006180B4F9161048438013A0807AE70000FA
:108330003F070020800A0020A4020020BC09002082
:10834000E2050020320100200D480021A32280F820
:108350002810C18381865030C2600E22028241F211
:108360006202426108220283418341F255528283B4
:108370009203C0E9081240F28E3282608162704737
:10838000300A00202DE9F0410546FBF7D9F9204CD1
:10839000204E074620686168421C8A4220D009B9F5
:1083A0003F281DD004EB0010AA7A05F10B010E3016
:1083B000F7F7E9FE2168686804EB0111886021681D
:1083C000A87A04EB0111888172B62068401C2060F5
:1083D000402801D30020206062B6307888B114E0D4
:1083E0003846FBF795F90A28D4D3706800F066FA8E
:1083F000002109A001F0C0FA70604FF0FF30BDE825
:10840000F08155203070F9F793FD0020F7E7000068
:10841000A8140020480800206465765F63616E310F
:108420000000000010B504000B462D4AC3F1000007
:1084300028D56442002B12DAA04207DA214600F068
:10844000E7FB32F81000C0F5404041E0014620460D
:1084500000F0DEFB32F8100000F5004038E0A342E7
:1084600008DA2146184600F0D3FB32F8100000F578
:1084700040402DE0204600F0CBFB32F81000C0F564
:10848000803025E0002B12DAA04207DA214600F006
:10849000BFFB32F8100000F5804019E0014620468D
:1084A00000F0B6FB32F81000C0F5004010E0A34227
:1084B00008DA2146184600F0ABFB32F81000C0F590
:1084C000804005E053B1204600F0A2FB32F81000D6
:1084D000B0F5004F01DDA0F5803010BD002010BDCB
:1084E000B0AF000840438013494300EBA1300022A5
:1084F0000302002B14DDB3F5001F01DC802001E036
:108500004FF4005093FBF0F1014401EBD17149109D
:10851000814206D0521CD2B20846062AF2D300E0AD
:108520000021C80000B2704702E008C8121F08C14D
:10853000002AFAD170477047002001E001C1121FE4
:10854000002AFBD1704700002DE9F047B94CBA482A
:1085500021880288511A89B20F297DD30088A4F19D
:108560003C052080288F08B1401E28872B78B34A0D
:10857000C3F3810001281ED0022821D0118BAD4801
:10858000B04EDFF8BC92407EB6F806C00027B1F5C9
:10859000926F1CD8142818D3782060764CF0100005
:1085A000F08040F26660A88123F001002870D77344
:1085B00089F8007018E0108B00EB4000C00302E067
:1085C000108BA1494843010CD9E7401C04E0B1F5E8
:1085D000216F09D910B1401E607605E02CF0100023
:1085E000F08043F001002870B5F90200B5F91430AD
:1085F0004143C3EBC303C1F38F31C3F3D10303EB97
:10860000510109B2A9829046128B4FF0805350431A
:10861000B5F91620C0F38F30C2EBC202C2F3D1020B
:1086200002EB500000B2E882AA6A42431213EA62E7
:1086300093FBF2F22A63854A1080A2680A44A26082
:10864000E1680144E160207C401CC0B2207407282E
:1086500002D942F3CF0000E0EAE02883C910698321
:10866000E760A76041F6C8012774884204DD2A8BC1
:108670007749B1FBF2F1E981C117890341EA9041E1
:10868000800342F69B420023F7F74CFDA88469481B
:108690002978A0F13C008B07B0F90600C1F38101F5
:1086A00000EB801202EB003242F30F3215D50129A4
:1086B00007D002290BD04EF6AC3141430914A180FA
:1086C00011E049F2586148430014A08020E04CF2C8
:1086D0000C3141430914A18026E001290ED0022962
:1086E00018D0A0806A845B4948430014A4F81E0097
:1086F000FAF764FB58480088C0B143E04AF2904161
:1087000041430914A1804BF2C821484300146884F6
:10871000E283EDE74CF6345141430914A1804DF654
:108720006C314143091469844C49DDE795F8200018
:1087300000BB88F80F7089F80070B5F91A00A0F531
:1087400014512C39B1F56E7F18D2617FF42912D9FA
:108750004349E8803F4AA1F8460050430014A880EE
:10876000A1F84400FF2085F8200081F828003D4949
:108770003C20087006E0491C617703E0607F08B187
:10878000401E6077B5F91A10B4F91E2036489142A0
:108790000DDDA27E7D2A08D9F28842F00802F2801F
:1087A000027822F0020202700EE0521C06E0A2F2F1
:1087B0003D12914208DAA27E12B1521EA27603E067
:1087C000F28822F00802F280B4F9042091420FDA14
:1087D000E17E3E2909D9F18841F01001F180277727
:1087E000017821F00201017013E0491CE17610E0EC
:1087F00002F23D12207F914208DD7D2804D9F088E5
:1088000020F01000F08004E0401C01E008B1401EA0
:108810002077B5F91810606908446061217E491C11
:10882000C9B221761F2903D94011A8836761277631
:10883000BDE8F0870C05002048070020A4020020B6
:108840003F070020000C002030330100700B002097
:1088500074E8260B188601004A070020E038010062
:10886000580E00203C070020E2050020024941F29A
:10887000F460886270470000D004002070B50D4C91
:10888000207828B1012808D0062505280FD10BE053
:108890000948F9F7C7FD012004E00748801DF9F7F2
:1088A000C1FD0520207070BDF9F7DCFD2570257035
:1088B00070BD000040070020B8AE00080A4A4FF023
:1088C000FF31B0EBA20F0CDA00280ADB0749096878
:1088D00051F820004068006900B100476FF00500C2
:1088E0007047084670470000040000007C08002024
:1088F00070B50A4DA86870B100240948AC60F8F75B
:10890000CFFC084804604460A0F5816004604460C6
:108910002C70002070BD6FF0040070BD480800206E
:1089200000640040A81400207FB505460024631EA3
:10893000244A4FF00050072D41D2DFE805F04004F3
:10894000111E21403C00814208D2D068202805DA5F
:108950001D4B43F82010401CD0600CE01C4627E063
:108960008142FBD210692028F8DA174B803343F894
:108970002010401C10610023F0E7F8F7A7FC17E077
:1089800000208DF80B000121ADF800000422ADF8A5
:108990000400ADF808008DF80C108DF80A00ADF851
:1089A0000220ADF806208DF80D106846F8F7CAFCD5
:1089B000204604B070BDBDE87F40FAF755BF1846A9
:1089C000F7E7000048080020B0180020F8B5414E35
:1089D000B06801287BD04048F8F762FC01210820EC
:1089E000FDF706F901210846FDF702F901214806C5
:1089F000FDF7E6F801214FF4EA10FAF74DFE4FF4C7
:108A00008070ADF8000003248DF802400420334D3F
:108A10008DF8030069462846FAF7ECFD6815ADF8B5
:108A200000008DF8024018208DF8030069462846A2
:108A3000FAF7E0FD14208DF8000002278DF8017090
:108A400000248DF8024001258DF803506846FCF79C
:108A500095FD13208DF800008DF801708DF80250FF
:108A60008DF803506846FCF789FD16208DF800004C
:108A70008DF801408DF802408DF803506846FCF7F0
:108A80007DFD17490120FFF74FFF16490120FFF731
:108A90004BFF15490120FFF747FF14490120FFF75D
:108AA00043FF13490120FFF73FFF00210320FFF799
:108AB0003BFFF8F7A1FB0F4804604460A0F581601C
:108AC0000460446034700020B560F8BDFFE74FF0EB
:108AD000FF30FAE74808002000640040000C014025
:108AE00020FF401820FF431820FF441820FF45189E
:108AF00020FF2518A81400202DE9F04781461E48C4
:108B000086B0174680680E46A0B14FF0FF381FB3FD
:108B10006846FAF7B7FE401C0ED00DF10B019DF828
:108B20000A208A464846019DF7F72DFB9DF80A402A
:108B30003D601DE06FF0040006B0BDE8F08700BFA7
:108B4000FAF792FE411C15D0A84213D16846FAF7F5
:108B500099FE0198A84201D04046EDE79DF80A2011
:108B600009EB04005146F7F70EFB9DF80A00044498
:108B7000B442E5D32046DFE7480800202DE9F0475E
:108B80000646224886B00024806888B1601E002A0C
:108B900010D012680192B2F1005F0BD2CF0801F041
:108BA00007054FF000084FF004094FF0080A17E0DE
:108BB0006FF0040006B0BDE8F08700BF8DF80AA092
:108BC0008DF8089006EBC4008DF809800168CDF897
:108BD0000B104068CDF80F006846FFF7D3FB641C0C
:108BE000BC42EBDB7DB18DF80A508DF808908DF812
:108BF000098006EBC4012A460DF10B00F7F7C3FA12
:108C00006846FFF7BFFB0020D4E7000048080020BB
:108C1000090A05D0B0FBF1F0FF2800D9FF2070470A
:108C200000207047D0E90021C368521A5A4301EB73
:108C3000A231816041607047B0F90020B0F90210A4
:108C4000B0F90630521A5A4301EBA23181804180BB
:108C50007047000030B5494B188849498A89801A05
:108C600085B24848484A0F2D047801F14C001DD3C5
:108C70001D888D81117A090713D5022C01D0434933
:108C800012E0434DB0F90210B5F90050A94205DCDD
:108C900002DA01F1020108E0458007E0A1F10201DA
:108CA00003E0022C02D13B4909884180B0F8401012
:108CB0001D88691A89B29C2949D31988A0F84010E7
:108CC000D16A0023B1F5804F31DB3349096DB1F52D
:108CD000405F2CDD314940F26665B1F91010A942C0
:108CE00012DD43F69915A94202DB40F2333108E068
:108CF00040F23335A1F26661694343F2333591FBAB
:108D0000F5F1A0F8441001E0A0F844302449B2F88D
:108D10000A510978C1F381012DB100BFB0F84410A8
:108D200001F21E511CE092F84A20032A10D0A0F84C
:108D30004430022C01D0A0F84430B0F95C10B0F9F6
:108D4000443001F114029A420DDAA0F85C2030BDE3
:108D5000012901D00229E1D1B0F8441001F23331E8
:108D6000A0F84410E5E703F11402914203DD143941
:108D7000A0F85C1030BDA0F85C3030BD4807002082
:108D8000000000203F070020A4020020CE040020A5
:108D9000CC040020C8040020380100203805002041
:108DA000D00400202DE9FC4101210220FCF708FF3E
:108DB00001211920FCF71CFF01213C48FAF76CFC4B
:108DC0004027ADF8007003248DF802400420384D90
:108DD0008DF8030069462846FAF70CFCE001ADF86F
:108DE00000008DF802401C208DF8030069462846DB
:108DF000FAF700FC4FF4E0712846FAF782FCA81558
:108E0000ADF800008DF8024010208DF8030069468F
:108E10002848FAF7EFFB4FF4A060FCF7E1FB1D20B8
:108E20008DF8040001268DF8056000258DF80650A8
:108E30008DF8076001A8FCF7A1FB1F498C20088072
:108E40001D494FF6FA702C3108806E20091F0880EA
:108E50001948143006801848083007801649203118
:108E60000D80154AD020121D1080134A45F2F300E0
:108E7000183210800A1F45F2500010800E4A4FF63B
:108E8000FF7038321080121D1080121D108041F2C8
:108E90001B10088000F012F8FAF71CFF064810308B
:108EA0000580001F0480BDE8FC810000000C1A0052
:108EB00000100140000C01400004004070B51D206E
:108EC000FCF72FFB2A4D40212846FAF711FC8400BD
:108ED00080212846FAF70CFC44EA4004A9152846EC
:108EE000FAF706FC0443E0B2224C84F83C00FAF79F
:108EF000A9FC0546052805D91F48C18841F0400155
:108F0000C18001E084F838501C48007A000703D57E
:108F100094F838001A490D5C4FF6FA702063E0624D
:108F2000A06260622062E061A06116486063002078
:108F30006064206584F83F0084F84000FAF730FC54
:108F4000A07AFF2811D0022084F83D000E48008846
:108F5000A0662846FBF720F9207820F00100207059
:108F6000BDE870401D20FCF7F2BA0120ECE70000DC
:108F70000010014038010020000C0020A402002055
:108F8000ACB80008DCFF0500240400402DE9F043E4
:108F90004D484E4902880B889A1A92B20F2A67D31D
:108FA000098801804A49C98B027D00EB4202918009
:108FB000017D491CC9B20175082959D300240475E3
:108FC0002246017D00EB4103491CB3F90430C9B2CC
:108FD00002EB630212B201750829F2D33D49047510
:108FE0003D4B4A8044800E789D895FEAC67C40F6FE
:108FF00038694FF0030714D0A2F22B5C42F6E85810
:10900000C44520D3A1F1020C26F00204ACF80020E4
:1090100047750C7040F22B54A24211DA45F004025D
:109020001EE046F001060E704A4507DD45F00102DC
:109030009A8126F002020A70477517E0447515E020
:1090400045F002020CE04A450CDA8775427D12B108
:10905000521E42750AE046F002020A7025F007022D
:109060009A8103E0837D2BB15B1E837540888880E5
:10907000BDE8F08342F6AA239A4222DAB1F904301D
:109080002BB941F2CD05AA4201DA4480EEE7134C38
:10909000920302EB843241F67244B2FBF4F214B252
:1090A0004FF4805502464480AC4200DA5580B2F954
:1090B0000240E41A04F5A374B4F5237FD6D84380A4
:1090C000D4E74FF48043FAE7940C002048070020CF
:1090D000A4020020E2050020000C0020C8F1FFFFE0
:1090E0002DE9F0416D4CDFF8B8E14FF0000594F840
:1090F0003410C80706D094F938104B42002958DDC7
:109100000E4657E0674884F83750A4F84250664A44
:1091100090F8380084F840009586CEF80450CEF8D8
:109120000850624E40F26663CEF80C50A4F87C30D2
:1091300036F810005E4E768830444FF6FF7606EA29
:10914000800024F8300B4FF0806044F8040CA3201A
:10915000208460845810A084E38440F69910208510
:10916000580060854FF48050A08541F23330E0858F
:1091700041F26660208641F69910608641F6CC4047
:10918000A0864FF40050E08642F23330208742F24E
:109190006660608742F69910A08742F6CC40E0876F
:1091A00082F8A15041F00100207184F84450BDE8DC
:1091B000F0811E4694F937004242002801DD07463F
:1091C00000E01746F61B012E0BD0002800DB0246FC
:1091D0005FFA82F684F8380094F84F00012805D031
:1091E00041E0002900DA1946CEB2F3E794F93930AC
:1091F0005942002B01DB184600E0084694F93A205A
:10920000C7B25042002A01DB944600E08446BC45C8
:1092100008DD002A00DA0246D7B2002B00DA0B463E
:10922000D8B207E0002B00DA0B46DFB2002A00DBE1
:109230001046C0B204EB4000B0F9501004EB4700F8
:1092400030F9502F11444910018084F84F5084F8B0
:109250003E5084F83D5084F83C5084F83B5084F8EC
:109260003A5084F8395004EB46007546B0F9500086
:1092700024F8420FBEF80410C82309B26422FDF797
:109280003DFA6860E968401AA9680844A860B5F921
:1092900000104843C013E860608788E7140C002082
:1092A000D005002038010020A4020020BEB800082C
:1092B0004C000020F0B4544890F83410C90776D020
:1092C000524990F84030002291F838108B426FD00C
:1092D0004F4CA0F872204F4DE65C04468E4294F944
:1092E000374002D0EE5C8E420FD1641C64B280F82D
:1092F0003740EB5C8B4202D1641C80F8374090F918
:1093000037300F2B1BDD0F2317E0434DEE5C434D31
:109310008E4202D0EE5C8E4211D1641E64B280F89F
:109320003740EB5C8B4202D1641E80F8374090F9E5
:1093300037406FF00E039C4201DA80F83730324B31
:1093400090F83F50393390F83740EC5490F83F3064
:109350005B1CDBB280F83F30062B01D380F83F2046
:1093600090F9394090F93B309C420ED190F93D4044
:10937000A3420AD190F93A4090F93C309C4204D182
:1093800090F93E40A34200D1012280F84F201F4AAD
:1093900080F8401090F937501378214A012D0DDDE7
:1093A00014465E07A46804D544F0080403E028E0EE
:1093B00015E024F00804946080F83510B5F1FF3F03
:1093C0000ADA5B07936802D523F0080301E043F053
:1093D0000803936080F83510F0BCFAF7E1B990F813
:1093E0004F1001290DD1B0F8721043F60953491CF2
:1093F00089B2A0F87210994203D9A0F8722080F8BF
:109400004F20F0BC70470000140C002038010020F1
:10941000A0B80008A6B80008B2B80008B8B800089C
:10942000A402002010B502884188B0F90830114428
:1094300009B281FB0313890B428041EA8341B0F9F1
:109440000420B0F9063082FB0332940444EA9332DC
:109450001144818010BD000030B52049204AB1F888
:109460006A301088C01A80B20F2836D31088A1F84D
:109470006A001C4D00204FF000432A5C940903D081
:109480000124B4EB921F24D1D20622D0164A52F8FE
:1094900020201268134C123434F81040224201EBA1
:1094A000000494F9722008D00A2A04DB0A6823FA1F
:1094B00000F4224308E0521C09E012F10A0F05DC17
:1094C0000A6823FA00F4A2430A6002E0521E84F8FC
:1094D0007220401CC0B21128CFD330BDE805002057
:1094E00048070020B4B30008B4B400082DE9F00721
:1094F0007A497B480A8903889A1A92B2082A75D356
:1095000000880881A1F12C0042890AB1521E4281D3
:10951000744A92F82820802A68D302F03F020A7029
:10952000C2890AB1521EC281B1F90620902A0CDB11
:109530008A46FF2A09D08146C089002856D16A4848
:1095400000230078092805D005E0BDE8F00763484E
:1095500000F0C4B90823654A92F8EE500DB143F00B
:1095600004036348817AC90701D043F00203D2F8AB
:1095700008C05FEA0C5101D543F0010317680021D0
:109580005C4EFC0302D596F8654004B18021C48886
:109590005FEA446801D541F040015FEA845801D593
:1095A00041F020015FEAC47801D041F01001007A57
:1095B000400701D541F008014F480078C00701D0AD
:1095C00041F00401A00601D541F001010020012D68
:1095D00000D1082096F870508DB992F84A20032ADD
:1095E00005D0022A06D0012A07D008E072E040F038
:1095F000030004E040F0020001E040F001007A07BF
:1096000001D440F02000CCF3C0020025CCF3002CA4
:10961000624502D13A0700D4042596F86F20012A4A
:1096200001D145F00105354A0027BC4612783E4677
:10963000C2F38102012A04D0022A04D0032A04D0F2
:1096400004E0022602E0042600E010262C4A64060C
:109650000ED5224C1C342478240609D514786406CF
:1096600006D4284A40F6CC44926D6243140C05E0BF
:10967000B2F8B62040F699146243940B4FF00808F4
:109680008AF80A804FF061088AF80B808AF80C305B
:109690008AF80D108AF80E008AF80F508AF81070B8
:1096A000270A4B4083F06901414069408AF81170F4
:1096B00079408AF81240614052468AF813C07140DE
:1096C0008AF8146051754FF4C871A9F80E10FF2084
:1096D000AAF80600BDE8F00770470000F406002075
:1096E00048070020E80500203F070020A4020020D2
:1096F000000C0020580E0020B00A0020D0040020EA
:1097000038010020540900205F48816941F0FC01C4
:1097100081614FF4A060FBF763FFFAF769FBF7F78D
:109720004FFAFBF7DDFD002158A000F025F95A495A
:109730000860FDF7F5F8FCF7E7FEFFF733FBFBF7F2
:109740003BFAFFF7BBFBFAF7C5FA544D4FF4005054
:10975000A5F81A01FCF7F4F8FCF7A8F800214FF47B
:10976000FA5340F2EE220020401C80B29842FBD314
:10977000491C89B29142F6D3494C002684F87260A4
:10978000F7F7AEF8F8F744FF42F2FF1020834FF4EA
:109790000950608342F22320A08342F2AE00A080F1
:1097A000F8F73CFCFEF740FC10223E493E48F6F735
:1097B000EAFC01F001FA3D4C3E4FE08820F0400009
:1097C000E0803B48017821F020010170FA20F88107
:1097D0004FF49670A5F84200FFF748F8364937482D
:1097E000FCF70FF83648FCF731F83648416A8847ED
:1097F0003548416B8847FEF7A7FD3448F9F7DAFA98
:10980000F8F73EFC32494220C8803249C8603248ED
:10981000F7F782FBA86820F48070A8603E71F7F724
:109820000BFCE088E0812089208260896082F9F762
:1098300043FEF9F79FFDFEF787FE01F03DF9FFF7C4
:10984000A5FB00F035FAFFF707FE00F0E7FFF9F798
:1098500085FBF8F73FFCFAF7BDFCFFF7FBF9FCF7D7
:1098600057FAFAF7DFF8FAF711F900F0B3F8FFF753
:109870003DFE1648F9F74AF900F0A6FAFCF788FE13
:10988000F9F7CEFACDE70000001002406465765F7C
:1098900063616E31000000004C080020A40200202B
:1098A00038050020580E002028060020000C00205B
:1098B000380100203C070020000A0020D0090020C9
:1098C0000C04002020000020CC0000203C0B0020D5
:1098D0003007002040040020B00B0020F0B52349E1
:1098E0000278B0F9064000231F4E31F81210FF2C09
:1098F00018D0B0F904701E4DBC4231DA00EBE40719
:1099000004F00704BF7AA7408478FFB23CB190F816
:1099100001C0ACF1010C64451FDA3C061DD455F8BA
:1099200022200DE056F82220116012498A79521C3B
:10993000D2B28A71022A02D38370C3808B71F0BDC8
:1099400011608178491CC9B2817042789142F6D386
:109950008370C188491CC180F0BD56F82220EFE712
:1099600055F822201160F4E794B50008C6B300084A
:109970003CB50008C80600202DE9F0410F4680469E
:109980000024124D124E08E0286850F824000168A7
:109990004046F6F70AFC38B1641CB4EBA60FF3DBC3
:1099A0006FF00100BDE8F081286850F8240040689D
:1099B000016829B13846884728B16FF00200F1E705
:1099C0006FF00500EEE72046ECE700007C08002081
:1099D00004000000F0B561486149B0F86C200B88C4
:1099E0009A1A92B29C2A7BD30988A0F86C105D4920
:1099F0005D4F91F82A1001F0070297F84A10022AE9
:109A000000D1491E594C80F83E104FF00203E28805
:109A10004FF00001550401D5012236E0A489E50686
:109A200001D5062231E0250701D508222DE0550693
:109A300003D44F4D2D78AD0601D5042225E0150540
:109A400001D5072221E0150601D50A221DE0950661
:109A500001D50C2219E0150701D50B2215E0550799
:109A600001D4D50501D510220FE0D50601D5052278
:109A70000BE0650703D4A50701D4E40702D080F802
:109A80006E3007E0920403D5032280F86E2001E0D7
:109A900080F86E10374A384C92F820E0324A251F81
:109AA000D2F808C02D4AB2F87060721C92B2BEF1B2
:109AB000000F0DD02CF4000CC7F808C090F86E70A1
:109AC000B7B11E2F1AD090F86F200AB325E007E037
:109AD0004CF40006BE60A0F870200A2A01D2236070
:109AE000F0BD142A01D22B60F0BDA0F87010F0BDBB
:109AF0002B60A0F8701080F86F10F0BD642E04D2B7
:109B0000A0F87020322AEED3E9E7A0F87010EAE757
:109B10007F1C80F86F70A0F8701090F86F20012AF9
:109B200010D0002AE9D0B0F87060761CB6B2A0F868
:109B300070601E2ED7D323603C2EDED9521E80F8D3
:109B40006F20D2E7B0F87020521C92B2A0F87020BB
:109B50002360C82AD1D980F86F10C6E7E805002035
:109B600048070020580E0020A4020020000C00200E
:109B700038010020D0040020141C0140F0B54548F5
:109B8000B0F84810491C89B2A0F8481002297DD3CA
:109B900041490024A0F848400A78404B042A5BD091
:109BA0004FF48041082A0BD0A0F10C02B2F900203A
:109BB0008A4200DA1146B3F984208A4200DA11465B
:109BC000374A12698A4200DA11B2418282881D8ABC
:109BD000C2EB8502334D12B22D78C5F381062D4DAF
:109BE00040F6D9467243B5F9765092126A43121381
:109BF000C26086681546C6EBC60642F3D102F6027D
:109C000002EBA6328260C66C1644C664B0F850708F
:109C10007F1CBFB2A0F85070B7F5806F04D3B612A6
:109C20000682A0F85040C464C66A891AA6EB46179B
:109C300040F2545207EB07174A43A7EBC61602EB54
:109C40004602466A32444262B3F93430B2EB034F03
:109C500006DD1A04426206E01349B1F90410AFE7C9
:109C6000002A00DA4462C162104990F83D2091F860
:109C700038108A420DD080F83D10B0F84210A0F89C
:109C80004410B0F84010A0F8421000E001E0A0F845
:109C90004050F0BD380500203F070020A4020020FE
:109CA000F80D0020D00400200C0E00203801002008
:109CB00015481649B0F85A200B889A1A92B20F2A02
:109CC00020D30988A0F85A10B0F900104FF4804250
:109CD000C1EBC12141F35131A0F86C100C490B7854
:109CE000A0F10C01022B06D1B1F90030934202DA47
:109CF0001B1D0B8000E00A800021A0F8601020F8F6
:109D00005C1F428070470000380500204807002093
:109D10003F0700204FF6FF7202EA800210F4404332
:109D200015480ED0B3F5804F14D0B3F5004F4FEA6D
:109D3000122216D0C2F5807330F813305B424B808C
:109D400005E0120A30F812304B80C2F5807230F80C
:109D500012000FE0120AC2F5807330F813304B8006
:109D600005E030F81230C2F580725B424B8030F86B
:109D70001200404208807047B0B10008104A518A72
:109D8000D08A928A16384639A2F1110200D549428A
:109D9000002A00DA52421144002800DA4042084406
:109DA000084943F6284300B2B1F936205A439213CA
:109DB00040F2D733584302EBA030C886704700000A
:109DC000A402002038050020F0B5904990480A8987
:109DD00003889A1A92B23E2A1ED30088088101F1A4
:109DE00038004FF4FA63428A9A4202D2521C4282ED
:109DF00000E04382874A92F82220802A0CD302F0A6
:109E00003F020A70B1F90620402A06DBFF2A04D07F
:109E1000C2883AB1521EC280F0BDBDE8F0407B4816
:109E2000FFF75CBD428A9A42F6D307784FF0010EE5
:109E30003A074FF0FF055BD5847A40F2DC526307A6
:109E400008D444F004038372C28081F80BE081F8E7
:109E50000AE04CE04378072B05D0032B03D0052BF9
:109E600001D0062B07D1660605D444F04003837267
:109E7000C280052239E0654A5FEA437C02F138027C
:109E80004FF42076127A0DD55FEAC26C0AD45FEAED
:109E9000446C07D442F0100202723A0628D4C680FD
:109EA000192222E0DF0709D0970707D4670605D4F7
:109EB00042F002020272C680042216E09F0709D512
:109EC000170707D4670605D442F008020272C6805D
:109ED00003220AE01B070BD5530709D4630607D4F6
:109EE00042F004020272C6800B22CA728A72CD80CE
:109EF000494AB2F92230B2F91A7003F23D14002235
:109F0000A74200DB0276414E444C06F13806A479A4
:109F1000B6895FEAC46C06F101064FF4C874B6B2A4
:109F200013D58681B6F57A7F05D9017A21F08001B3
:109F300001728281F0BD037A1E06FBD4828143F058
:109F400080020272C480112035E09F4216DA037E3F
:109F5000052B13D28681B6F5487F04D98281027A17
:109F600022F040020272027A5606E3D45B1C0376AA
:109F700042F040020272C48002201CE0284B1C897F
:109F8000C4F3C006C4F3002740F2EE24BE4216D14B
:109F90001E78360713D4427E012ACBD1428BB2F50C
:109FA000167F02D2521C4283F0BD827A42F0020236
:109FB0008272C4800F20C8728872CD80F0BD93F881
:109FC00011714FF40046012F18D1164F41F6583C3D
:109FD0007F6C674512DD83F810E1134B1E60C38A66
:109FE000A34202D25B1CC382F0BD4FF4FA73C3805C
:109FF0001C23CB728B72CD80C282F0BDC2820A4814
:10A0000083F81021001F0660F0BD0000D806002074
:10A0100048070020E8050020D0040020000C0020A4
:10A02000A402002038010020140801402DE9F05F4F
:10A03000DFF8F4B3FD48FE4C9BF81830011D0A1DF3
:10A04000012B5DD0B4F85E300380B4F86000088066
:10A05000B4F862001080FDF731FBDFF8D883F64DCD
:10A0600049F2CD32B8F91E10A983B8F9200043F6A1
:10A07000CC4C01EB400050430014E883B5F922308A
:10A08000B5F9206000FB03F201FB062242F38F3298
:10A090006A82B5F91870704307FB0CF740F2333C45
:10A0A000BF1302FB0CF207EBA23201FB13002A8361
:10A0B00040F38F30A882B5F91A1043F6AE725143BF
:10A0C00000EB0012891302EB8010DC4E01EBA03094
:10A0D000DB4F6883706C3860396938468847D949E6
:10A0E000388948800846FDF7CBFBD74F4FF0010A6F
:10A0F000387808280DD0698F298204283BD01BE0CE
:10A10000B4F864300380B4F866000880B4F86800DE
:10A11000A0E7CE4890F93710491C022929D890F8B9
:10A12000741019B1B5F85A00288205E0698F2982A8
:10A13000A5F85A1080F874A0B5F91410B5F90A0002
:10A14000C34AF8F787FBE862B4F91A11884204DDC4
:10A15000BF48E962027C91408162387804280ED0C1
:10A16000BB4AB5F91210B5F90800303AF8F772FB9E
:10A1700008E0688FD8E7D8F824000014E862B07AC5
:10A18000E8B3B448A862AC4DB14E443EA86A306012
:10A19000E86A706030461035FBF796FD2888A5F117
:10A1A0004C01FFF7B7FDA5F15C08DFF8AC92D8F8D9
:10A1B0001010C8F86C10B5F91010B068B5F912207D
:10A1C00000FB01F7F368504303FB127646F38F3729
:10A1D00003FB010040F38F36AF87EE87A9F80270CA
:10A1E0004D46A9F804604846FDF790FF287F08F126
:10A1F0001405012835D070424110698000E02DE03F
:10A200004DF6B35047433A142A804046A8F8006000
:10A210008B184380891AA8F804104FF0000984F8BD
:10A220000C90B8F90030002B01DD84F80CA0B8F9CF
:10A230000200002802DD217B891C2173B8F904206B
:10A24000002A02DD217B091D2173217B07291FD2F2
:10A25000DFE801F01E1A33172F1C31004FF4AF70E6
:10A2600090E7B9F920304DF6B35259424910698050
:10A27000B9F91E00504302142A804046A8F8003065
:10A28000C6E784F80DA003E0022100E0032161731A
:10A29000DFF8A4A1714E724F9AF800100129617B7A
:10A2A0000DD007297ED2DFE801F07DFDFCFBFAF935
:10A2B000F8000421EBE70521E9E70621E7E7072994
:10A2C000F0D2DFE801F06F042F5D84D6F000014684
:10A2D0001846FBF77DFA2860B5F9020040F6815177
:10A2E000484380136880B5F9001040F6815251430D
:10A2F000891329804218A2F68152B8F80A305242D6
:10A30000C3EB620212B2A8F80820002A01DCA8F808
:10A310000890B8F80820A4F862201044A4F860005F
:10A32000084474E1404201B2504200B2FBF750FAD7
:10A330002860B5F9020040F68151484380136880D7
:10A34000B5F9001040F68152514389132980421813
:10A35000A2F68152B8F80A305242C3EB620212B23E
:10A36000A8F80820002A01DCA8F80890B8F808200E
:10A3700075E13046F6F782FC01231A460721D7E043
:10A3800019461046FBF724FA2860B5F9020040F69A
:10A390008151484381136980B5F9000040F681522C
:10A3A000504300E0CFE0801328800A18A2F68152C3
:10A3B000B8F80A305242C3EB620212B2A8F8082081
:10A3C000002A01DCA8F80890B8F8082074E1594286
:10A3D000404209B200B2FBF7FBF92860B5F9020070
:10A3E00040F68151484381136980B5F9000040F679
:10A3F00081525043801328800A18A2F68152B8F87F
:10A400000A305242C3EB620212B2A8F80820002AB6
:10A4100001DCA8F80890B8F80820A4F85E201144E0
:10A42000A4F8601008447DE13C0B0020342C01406E
:10A43000A4020020380500204C0000203801002034
:10A4400040040020FC0300203F070020140C0020E3
:10A45000000A0020A2FEFFFF700B00200024014034
:10A46000002801403046F6F709FC01231A46052171
:10A470005EE01146FBF7ACF92860B5F9020040F642
:10A480008151484380136880B5F9001040F681522D
:10A49000514389132980421806E07CE150E121E113
:10A4A000F2E0C2E095E016E0A2F68152B8F80A3078
:10A4B0005242C3EB620212B2A8F80820002A01DC63
:10A4C000A8F80890B8F80820A4F860201044A4F870
:10A4D0005E00084451E1504201B2584200B2FBF71D
:10A4E00077F92860B5F9020040F68151484380139E
:10A4F0006880B5F9001040F68152514389132980D4
:10A500004218A2F68152B8F80A305242C3EB6202F6
:10A5100012B2A8F80820002A01DCA8F80890B8F8C0
:10A52000082052E13046F6F7A9FB01231A4606211E
:10A530003846F6F7A3FB01213046F6F715FB01215B
:10A540003846F6F711FBBAF80800ABF80000BAF885
:10A550000A00ABF80200BAF81000ABF80400554648
:10A560005E46AB48F8F734FBB4F85E00F188084467
:10A57000A4F86400B4F8600031890844A4F86600C7
:10A58000B4F8620071890844A4F86800317EA148DB
:10A59000012978D034F85E1F018061884180A1884C
:10A5A00081809C49028808310A8042884A808088DC
:10A5B00088809848896A0830884795F83E000028C6
:10A5C0007ED0F7F74FFF15F83E0F401E2870BDE80C
:10A5D000F09F01461846FBF7FBF82860B5F902002A
:10A5E00040F68151484381136980B5F9000040F677
:10A5F0008152504380130A18A2F6815252425208E7
:10A6000028801144A4F86220A4F860100844A4F83B
:10A610005E0000213046F6F7A7FA00213846F6F72B
:10A62000A3FA01231A460621A3E6404201B2504292
:10A6300000B2FBF7CDF82860B5F9020040F6815171
:10A64000484380136880B5F9001040F681525143A9
:10A6500089134218A2F68152524229805208A4F866
:10A6600062201044A4F85E000844A4F860000021B1
:10A670003046F6F779FA00213846F6F775FA0123E5
:10A680001A46052175E6B4E019461046FBF7A0F816
:10A690002860B5F9020040F6815148438113698072
:10A6A000B5F9000040F68152504380130A18A2F613
:10A6B0008152524228805208A4F85E20114400E0E2
:10A6C0009AE0A4F862100844A4F860000021304623
:10A6D000F6F74AFA00213846F6F746FA01231A46F9
:10A6E0000721BFE65942404209B200B2FBF770F8B9
:10A6F0002860B5F9020040F6815148438013688014
:10A70000B5F9001040F68152514389134218A2F660
:10A710008152524252082980A4F85E201044A4F8C5
:10A7200060000844A4F8620000213046F6F71CFAE5
:10A7300000213846F6F718FA01231A46062191E659
:10A740001146FBF745F82860B5F9020040F6815143
:10A75000484381136980B5F9000040F681525043A7
:10A7600080130A18A2F681525242520828801144DE
:10A77000A4F86020A4F85E100844A4F86200002148
:10A780003046F6F7F1F900213846F6F7EDF90123E6
:10A790001A460521C6E6504201B2584200B2FBF704
:10A7A00017F82860B5F9020040F68151484380133C
:10A7B0006880B5F9001040F6815251438913421860
:10A7C000A2F68152524229805208A4F86020104417
:10A7D000A4F862000844A4F85E0000213046F6F7B1
:10A7E000C3F900213846F6F7BFF901231A460721BD
:10A7F00098E634F8641FCFE607480088A0F5D041FA
:10A8000068393FF4E4AEBDE8F05FF8F78FBC0000B4
:10A810003C0B002018000020182C01402DE9F041CD
:10A82000974C9848B4F862100288511A89B20F29DF
:10A830006FD30088A4F8620093480088DFF84C8248
:10A84000C0074FF000054FF0010741D08E4AD4E910
:10A850000C1024321388B1EB530F02D21288511A14
:10A8600008444FF4F371884200D208468849B1FB8E
:10A87000F0F0616CC1F35101084406466064F5F7DD
:10A88000DAFD0022834BF5F742FD4FF04042824B48
:10A89000F5F73DFD0E22F5F7A9FDF5F703FEA4F847
:10A8A000AC0094F86D00401CC0B284F86D0008281C
:10A8B00034D3734898F84A20001F03789A4201D095
:10A8C00002704580754A1378754A23B1458021E0AE
:10A8D0006564256568E0D8F89810A1F5FA618E42A4
:10A8E00011DDE16D8B1C9E4205DDB0F902100A29D5
:10A8F0000DDA491C06E08E4205DAB0F90210002993
:10A9000008DD491E4180B0F902000A2802DB1770F9
:10A9100001E0B0E01570E66584F86D5061484FF4D1
:10A92000A5420178C1F38103012B59D044F2506153
:10A930002181A4F8A820B0F9243089B24B439B139D
:10A94000A4F8A430B0F90E00D4F850C07043B0FBA6
:10A95000F1F35549CCEBCC0C4FEACC2C0988C3F36E
:10A96000D10303EB9C33B0032365B0FBF1F14F4BF4
:10A97000C908B3F846C0CCEBCC0C4FEACC2C01EBA9
:10A980009C31A3F84610F117890341EA9641002350
:10A99000F5F7C8FBB4F8AA10C1EBC101C902C008A1
:10A9A00000EB9130A4F8AA00616C206F0844206786
:10A9B00094F87420521CD2B284F87420082A05D36B
:10A9C000C008A4F8760084F874502567384A394ED8
:10A9D000D388580631D498F80F00022803D02AE013
:10A9E00045F6C051A4E7B06840F69916B04222DDA2
:10A9F00094F8380094F88E60B0420CD084F88E0041
:10AA000094F83D0000F00106C0F34000864202D1F8
:10AA1000A4F88A5005E0B4F88A0040F6C416B042A3
:10AA200005D2B4F88A00401CA4F88A0005E043F07F
:10AA30008000D08001E0A4F88A50114894F83F309B
:10AA4000B8300C2B01D2C57400E0C774194A41F22A
:10AA5000482C41F2504692F83C400C4A0C2BB2F87C
:10AA600086200AD3614508DB012C06D0B14202DD05
:10AA7000002A00D18774BDE8F0818574FBE70000EF
:10AA8000380100204807002000040040A4020020F4
:10AA90004564BD0100209C40133B3340FA03002075
:10AAA000FB030020D004002030010020300A0020E9
:10AAB000000C00203805002070B5394C3948218839
:10AAC0000288511A89B23E294DD30088364E208023
:10AAD0003649307806F1140518B3488B8000288079
:10AAE000E96828468847B5F904003149FCF799FD23
:10AAF000304A60804FF48045D3884FF000015E07F4
:10AB000037D4B0F5DC5F2FDDE079401CC0B2E071D6
:10AB10000A283ED343F4004040F00400D080A160F6
:10AB200036E0888B204A8000121D1080888B8000C0
:10AB30005080888B800000B290804A8B92002A80DF
:10AB40004A8B92006A80498B8900A98018497C3120
:10AB5000FCF767FDA080B5F904001549FCF761FD1D
:10AB600060800120307070BD23F40040A560D0806B
:10AB70000EE043F4004343F00403A160D380B0F53A
:10AB8000B45F06DC23F4004020F00400D080A56010
:10AB9000E171D4E90201884200DB0846206170BD02
:10ABA000F80D00204807002094060020A402002091
:10ABB000A8B70008000C002005494FF48040C86089
:10ABC000886008610348C18821F48271C1807047A0
:10ABD000F80D0020000C00202DE9F041384C394ED2
:10ABE000394F207841F23331C2074FF000050CD0C5
:10ABF000A28962B394F90700002800DA4042C0B28B
:10AC0000032829D240F2AE702AE0A570E5732F4ADE
:10AC1000E571A58192F83830237220F00800A180F8
:10AC200040F002002070BD867560B560F560116D62
:10AC3000490005D041F68461A18140F010002070E8
:10AC4000C0B240F0010020706574BDE8F0816581FC
:10AC500020F01000207015E0042803D240F65100C7
:10AC600060810FE0052802D240F69910F8E740F61F
:10AC7000CC42062803D3072801D3082801D26281D9
:10AC800000E0618197F8A10098B9B088102301B263
:10AC9000B4F90A003622FBF731FD7060F168401A02
:10ACA000B1680844B060B6F900104843C013F060C2
:10ACB000B886B88E10B10120A070C6E7A570C4E7B1
:10ACC0000C0E0020B8060020A4020020380100204D
:10ACD0002DE9F041554C2678F0077CD05448217A74
:10ACE000544D90F8380081427BD0534A2346DFF818
:10ACF0004CC1575C93F90E2093F90730874203D07B
:10AD00001CF80170874213D146F002065B1C2670C6
:10AD10005BB2E3711CF80110814201D15B1CE3714D
:10AD200094F90710062901DD0621E171521C1CE08F
:10AD3000434F17F801C0434F844503D017F801C0B3
:10AD4000844513D126F002065B1E26705BB2E371C8
:10AD5000795C814201D15B1EE37194F907306FF099
:10AD600005018B4200DAE171521EA273207294F940
:10AD700007108A1C042A02D941F68462A2812C4A57
:10AD8000012912780ADD2B4B56079B6802D543F048
:10AD9000080301E023F00803AB606070B1F1FF3FEE
:10ADA00009DA5107A96802D521F0080101E041F054
:10ADB0000801A9606070F8F7F3FCA078012810D1B1
:10ADC00021488068A3280CDA94F90700022803DDE3
:10ADD0000220E07105E01EE06FF00101884200DA18
:10ADE000E171A089002630B1401E0004000CA08152
:10ADF00001D1E671A673E87B04280CD0B5F93410B4
:10AE0000512341220020FBF779FCA886002802D1BB
:10AE1000E07B10B1A670BDE8F0810C4806700C48CC
:10AE20000670207820F001002070F4E70C0E00205E
:10AE300038010020A4020020A0B80008A6B800082D
:10AE4000B2B80008B8B80008380500205C07002038
:10AE50003F070020F0B415460D4A0E464FF0FF3173
:10AE6000B0EBA20F12DA002810DB0A49096851F88A
:10AE70002000406844682CB129463046A446F0BC06
:10AE80001A4660476FF00500F0BC70470846FBE7C4
:10AE9000040000007C080020173E573CBB3A3E39B6
:10AEA000DD379436613541343333353244316130E6
:10AEB0008A2FBD2EFB2D412DCC1C5858586899194E
:10AEC000585858683313005695130054B61300525F
:10AED0005A140050FD14004EA115004C4516004AAE
:10AEE000761600486C17004672180044BA190042E2
:10AEF000741B0040911D003EB420003C9F22003A8C
:10AF0000E1220038532300368B240034812500329F
:10AF10002B2700302028002E5829002CB02A002A88
:10AF20009B2C0028D22D00267C2F002426310022C5
:10AF300002330020FD34001E5C37001CCC3C001A9C
:10AF4000873E0018BE3F001600400014004000126B
:10AF5000004000100040000E0040000C0040000ABD
:10AF600000400008004000060040000400400002CD
:10AF70000040000001020304050005000102030473
:10AF80000104000305020000F0010000360100008A
:10AF9000F8000000BA0000007C0000007C00000007
:10AFA0007C000000C91C9C19991CCC199C1CC91957
:10AFB0000000290052007B00A400CC00F5001E0117
:10AFC000470170019901C201EA0113023C026502C6
:10AFD0008E02B602DF020803300359038203AA037C
:10AFE000D303FB0324044C0475049D04C504EE0440
:10AFF00016053E0567058F05B705DF0507062F0611
:10B0000057067F06A706CE06F6061E0746076D07FB
:10B010009507BC07E4070B08320859088108A808FF
:10B02000CF08F6081D0944096A099109B809DE0923
:10B03000050A2B0A520A780A9E0AC40AEA0A100B69
:10B04000360B5C0B820BA80BCD0BF30B180C3E0CD4
:10B05000630C880CAD0CD20CF70C1C0D410D650D6A
:10B060008A0DAF0DD30DF70D1C0E400E640E880E29
:10B07000AC0ECF0EF30E170F3A0F5E0F810FA40F19
:10B08000C70FEA0F0D103010531075109810BA103A
:10B09000DD10FF102111431165118711A911CA118B
:10B0A000EC110D122E12501271129212B312D41210
:10B0B000F41215133613561376139613B713D713CA
:10B0C000F61316143614561475149414B414D314B9
:10B0D000F214111530154E156D158C15AA15C815DD
:10B0E000E7150516231641165F167C169A16B71635
:10B0F000D516F2160F172C17491766178317A017C6
:10B10000BC17D917F51711182E184A186618811888
:10B110009D18B918D418F0180B19261942195D1981
:10B1200078199219AD19C819E219FD19171A311AAF
:10B130004C1A661A801A991AB31ACD1AE61A001B0D
:10B14000191B331B4C1B651B7E1B971BAF1BC81B9E
:10B15000E11BF91B121C2A1C421C5A1C721C8A1C63
:10B16000A21CBA1CD21CE91C011D181D301D471D54
:10B170005E1D751D8C1DA31DBA1DD01DE71DFD1D77
:10B18000141E2A1E401E571E6D1E831E981EAE1EC4
:10B19000C41EDA1EEF1E051F1A1F2F1F451F5A1F40
:10B1A0006F1F841F991FAE1FC21FD71FEC1F0020E7
:10B1B00000006400C9002D019201F7015B02C0028A
:10B1C00024038903ED035204B6041A057F05E30541
:10B1D0004706AB060F077307D7073B089F0802090E
:10B1E0006609C9092D0A900AF30A560BB90B1C0C03
:10B1F0007F0CE20C440DA60D090E6B0ECD0E2F0F29
:10B20000900FF20F5310B41015117611D711381298
:10B210009812F8125813B81318147714D614351559
:10B220009415F3155116B0160E176B17C91726187B
:10B230008318E0183D199919F519511AAD1A081B10
:10B24000631BBE1B181C731CCD1C261D801DD91D25
:10B25000321E8A1EE31E3B1F921FEA1F41209820C8
:10B26000EE2044219A21EF2145229922EE22422309
:10B270009623E9233C248F24E22434258525D725F1
:10B2800028267826C82618276827B727062854288E
:10B29000A228EF283D298929D629222A6D2AB82AF1
:10B2A000032B4D2B972BE12B2A2C722CBB2C022D20
:10B2B0004A2D912DD72D1D2E632EA82EEC2E302F2A
:10B2C000742FB82FFA2F3D307F30C030013141311B
:10B2D0008131C13100323F327D32BA32F7323433FC
:10B2E0007033AC33E73322345C349534CE340735D5
:10B2F0003F357735AE35E4351A3650368536B936B2
:10B30000ED36203753378637B737E937193849389C
:10B310007938A838D738053932395F398B39B73998
:10B32000E2390D3A373A603A893AB23ADA3A013BB1
:10B33000283B4E3B733B983BBD3BE03B043C263CEB
:10B34000483C6A3C8B3CAB3CCB3CEA3C093D273D4E
:10B35000443D613D7D3D993DB43DCE3DE83D013EDE
:10B360001A3E323E493E603E763E8C3EA13EB53EA0
:10B37000C93EDC3EEF3E013F123F233F333F433F98
:10B38000513F603F6E3F7B3F873F933F9E3FA93FCA
:10B39000B33FBC3FC53FCD3FD53FDC3FE23FE83F39
:10B3A000ED3FF13FF53FF93FFB3FFD3FFF3FFF3FE3
:10B3B000FF3F0000E0203420002020E02020202358
:10B3C0003720262021000080020004000800100021
:10B3D000000200040008040000020004000800103D
:10B3E00000200040008004000000008000000040B9
:10B3F0000000002000000010000000080000000411
:10B400000000000200000001000080000000400079
:10B4100000002000000010000000080000000400F0
:10B420000000020000000100008000000008014050
:10B43000000C0140000C0140000C0140000C0140D8
:10B44000000C0140000C0140000C014000100140C4
:10B4500000100140001001400010014000100140A8
:10B460000010014000100140001001400014014094
:10B4700004080140040C0140040C0140040C01408C
:10B48000040C0140040C0140040C0140040C014078
:10B490000410014004100140041001400410014058
:10B4A0000410014004100140041001400410014048
:10B4B0000414014008080140080C0140080C014038
:10B4C000080C0140080C0140080C0140080C014028
:10B4D000080C01400810014008100140081001400C
:10B4E00008100140081001400810014008100140F8
:10B4F00008100140081401400C0801400C0C0140E8
:10B500000C0C01400C0C01400C0C01400C0C0140D7
:10B510000C0C01400C0C01400C1001400C100140BF
:10B520000C1001400C1001400C1001400C100140A7
:10B530000C1001400C1001400C1401401008014097
:10B54000100C0140100C0140100C0140100C014087
:10B55000100C0140100C0140100C01401010014073
:10B560001010014010100140101001401010014057
:10B570001010014010100140101001401014014043
:10B5800000000000000000000000000000000000BB
:10B590000000000014080140140C0140140C01408C
:10B5A000140C0140140C0140140C0140140C014017
:10B5B000140C0140141001401410014014100140FB
:10B5C00014100140141001401410014014100140E7
:10B5D000141001401414014000000000000000009D
:10B5E000000000000000000000000000FFFFFF0F4F
:10B5F0000FFFFFFFFFF0FFFFFF0FFFFFFFFFF0FF59
:10B600000FFFFFFFFFF0FFFFFF0FFFFFFFF0FFFF48
:10B610000FFFFFFFFFF0FFFFFF0FFFFFFFFFF0FF38
:10B62000FFFF0FFFFFFFFFF0FFFFFF0FFFF0FFFF28
:10B630000000004040000000000400000040000046
:10B640000000040040000000000400000040000072
:10B650000004000040000000000400000040000062
:10B660000000040000004000000000040000004052
:10B6700000040000000000808000000000080000BE
:10B6800000800000000008008000000000080000AA
:10B69000008000000008000080000000000800009A
:10B6A000008000000000080000008000000000088A
:10B6B00000000080000800000000002020000000C2
:10B6C0000002000000200000000002002000000036
:10B6D0000002000000200000000200002000000026
:10B6E0000002000000200000000002000000200016
:10B6F00000000002000000200002000000000060C6
:10B70000600000000006000000600000000006006D
:10B71000600000000006000000600000000600005D
:10B72000600000000006000000600000000006004D
:10B73000000060000000000600000060000600003D
:10B74000008002000400080010000002000400084D
:10B7500004000002000400080010002000400080E7
:10B7600004000000FF7FFFFFFDFFFFFFFBFFFFFF67
:10B77000F7FFFFFFEFFFFFFFFFFDFFFFFFFBFFFFF7
:10B78000FFF7FFFFFBFFFFFFFFFDFFFFFFFBFFFFDB
:10B79000FFF7FFFFFFEFFFFFFFDFFFFFFFBFFFFF31
:10B7A000FF7FFFFFFBFFFFFF401FFC02001E5A034D
:10B7B000C01CC403801B3C04401AC6040019630566
:10B7C000C01717068016E4064015CD070014D708E9
:10B7D000C012050A80115B0B4010DD0C000F900EAB
:10B7E000C00D7510800C9012400BE014000A651714
:10B7F000C0081C1A8007FD1C400600200005182305
:10B80000C003372680024E2940014C2C0000242F13
:10B81000C0FEC73180FD2E3400FB2D3880F81C3B64
:10B8200000F6003C8025151A40249A1B00231E1D9B
:10B83000C021B81E80205D20401F0C22001EC223A4
:10B84000C01C7E25801B3327401AFB280019B72A0D
:10B85000C0176D2C8016192E4015B92F00144731D2
:10B86000C012C9328011353440108B35000FCA36F2
:10B87000C00DF037800CFE38400BF439000AD23A84
:10B88000C008983B8007473C4006E13C0005673D07
:10B89000C003DA3D80023E3E4001923E0000143F6C
:10B8A000010203040500020304050001030405006E
:10B8B000010205000102030404050001020355050D
:10B8C0000010AA1A55250030AA3A0000AA0A5515F8
:10B8D0000020AA2A5535FF3F6465765F63616E31AB
:10B8E00000000000CD8900087D8B0008F98A00085F
:10B8F00029890008F188000800000000D8B8000875
:10B90000E4B8000828B90008000000208C080000F6
:10B910000007000854BA00088C0800203C150000FD
:10B9200038850008FCB8000801441381401B0895C5
:10B9300004211355152A4006190801A713CB5A1BD9
:10B9400008F1041AEB04012423286E4201170206B1
:10B9500004050103148020FF8BAA0A0201A415AA82
:10B960000A551500085920AA2A5535FF3F0731030B
:10B97000010504060203127C1573FFFF04FF80809B
:10B9800001012D025F6402130A13258C5208120173
:10B99000100C0504060203010103070505280B012D
:10B9A0000203040206070303040C3D07060405090D
:10B9B000191F191904310506060B14AA1A02312E93
:10B9C00040FD3969260211042F405F020C26405BBE
:10B9D000262ACD55155515123902017F0316D007B9
:10B9E0001AFF01013B0261AA0C10080108A8349952
:10B9F0003F33132594391CA9100916E8912203122C
:10BA0000100A17401C12600A16901B011AA2646BE0
:10BA1000398C94012199D0019A5A14021AC802CB88
:10BA2000D007023A19164902892612C8DA01DA1A31
:10BA3000FF01C1227D130D0212103AFA0812081CF0
:10BA4000F401010812062BE8031012021B24B91599
:04BA5000B100000041
:020000040800F2
:10FC00004A46545A594D46312D4E3330202020203B
:10FC1000050406020301AA0AAA0AAA0AAA0AAA0A4B
:10FC2000AA0ADE3F00100000FF0131000301664612
:10FC300000400040513800400040004000400101B9
:10FC4000004000407A3B082708270827FF0033338D
:10FC50000201401F00016626B81E6626FFFFFFFF57
:10FC6000FFFF01010100010000000300000202008B
:04FC70000000AA5591
:04000005080000ED02
:00000001FF
